:10000000A2C30000D8C30000D6C30000D4C30000C0
:10001000D2C30000D0C30000CEC30000CCC3000098
:10002000CAC30000C8C300000C94D3310C94BB3287
:100030000C948831C0C30000BEC30000BCC30000E4
:10004000BAC30000B8C30000B6C30000B4C30000C8
:10005000B2C300000C94AF31AEC30000ACC30000CB
:10006000AAC30000A8C30000A6C30000A4C30000E8
:10007000A2C30000A0C300009EC300009CC30000F8
:100080009AC3000098C3000096C3000094C3000008
:1000900092C3000090C300008EC300008CC3000018
:1000A0008AC3000088C3000086C30000050109025E
:1000B000A10185020901A1000509190129081500FE
:1000C0002501950875018102050109300931158165
:1000D000257F95027508810609381581257F9501D0
:1000E00075088106050C0A38021581257F95017572
:1000F000088106C0C005010980A101850319012AF4
:10010000B700150126B700950175108100C0050CD8
:100110000901A101850419012AA002150126A002E6
:10012000950175108100C005010906A1018506052C
:100130000719E029E71500250195087501810205D9
:1001400007190029EF1500250195F07501810205B9
:10015000081901290595057501910295017503910D
:1001600001C00660FF0961A1010962150026FF00B8
:100170009520750881020963150026FF00952075FA
:10018000089102C005010906A101050719E029E748
:1001900015002501950875018102950175088101F9
:1001A0000507190029FF150026FF0095067508812F
:1001B000000508190129051500250195057501910E
:1001C00002950175039101C00000000000000000CD
:1001D000000000000000000000000000000000001F
:1001E0000000000000000000000000007E0F00D4AE
:1001F000FFFFFFC7000000780000000000000000C3
:100200002A2B280000000000000000000000000071
:1002100000000029000000002C1E3420212224347C
:100220002627252E362D3738271E1F20212223244E
:1002300025263333362E37381F0405060708090AEA
:100240000B0C0D0E0F101112131415161718191A86
:100250001B1C1D2F3130232D350405060708090A04
:100260000B0C0D0E0F101112131415161718191A66
:100270001B1C1D2F3130354C0902BF00050100A0A9
:10028000FA09040000010301010009211101000124
:10029000224400070581030800010904010002034C
:1002A000000000092111010001222200070582033C
:1002B00020000107050303200001090402000103D7
:1002C00000000009211101000122B6000705840386
:1002D000200001080B0302010100000904030000D3
:1002E00001010000092401000109000104090404BE
:1002F000000201030000072401000141000624025E
:100300000101000624020202000924030103010284
:10031000010009240302040101010009050602404D
:1003200000050000052501010109058502400005C1
:10033000000005250101031201000200000008551C
:10034000A401000100010203011C037600690061A1
:10035000006C003A00660036003400630032006230
:10036000003300630000000A035300500049004EB0
:10037000000000160344004D0051002000440065B9
:10038000007300690067006E000000040309042484
:100390000021001E002700A800250022001F0020C9
:1003A00078A8002600230020002800A800240021AF
:1003B000001E002700A800250022001F002078A8AA
:1003C000002600230020002800A800A900AA00A9F8
:1003D00000AA00A900AA00A900AA00A900AA00A9D1
:1003E00000AA002223252628292A2C2D2F3032333B
:1003F0003536383A3B3D3E4042434547494A4C4EEC
:100400005051535557595A5C5E6062646668696B17
:100410006D6F71737577797B7D7F81838587898A1D
:100420008C8E90929496989A9C9E9FA1A3A5A7A823
:10043000AAACAEAFB1B3B4B6B8B9BBBCBEBFC1C253
:10044000C3C5C6C7C9CACBCCCDCED0D1D2D2D3D4E6
:10045000D5D6D7D7D8D9D9DADADBDBDBDCDCDCDC04
:10046000DCDDDDDDDDDCDCDCDCDCDBDBDBDADAD9D2
:10047000D9D8D7D7D6D5D4D3D2D2D1D0CECDCCCB54
:10048000CAC9C7C6C5C3C2C1BFBEBCBBB9B8B6B472
:10049000B3B1AFAEACAAA8A7A5A3A19F9E9C9A9802
:1004A000969492908E8C8A89878583817F7D7B79D3
:1004B000777573716F6D6B6968666462605E5C5AB4
:1004C0005957555351504E4C4A4947454342403E77
:1004D0003D3B3A3836353332302F2D2C2A29282609
:1004E000252322FFAA7F55400001010101010101DE
:1004F00001010202020202020202020303030303D9
:1005000003030304040404040404050505050506A7
:100510000606060607070707070808080809090965
:10052000090A0A0A0B0B0B0C0C0C0D0D0D0E0E0E0E
:100530000F0F0F101011111112121313141415159F
:1005400016161717181819191A1A1B1B1C1D1D1E11
:100550001E1F202021222223242425262627282965
:10056000292A2B2C2D2D2E2F303132323334353693
:100570003738393A3B3C3D3E3F4041424344454693
:100580004748494A4C4D4E4F50515354555658596F
:100590005A5B5D5E5F616264656668696B6C6D6F16
:1005A0007072737577787A7B7D7E80828385878889
:1005B0008A8C8E8F91939596989A9C9EA0A2A3A5C3
:1005C000A7A9ABADAFB1B3B5B7BABCBEC0C2C4C6C4
:1005D000C9CBCDCFD1D4D6D8DBDDDFE2E4E7E9EB80
:1005E000EEF0F3F5F8FAFDFF1E0F0500047F3F1F44
:1005F000643214643214783C1E1E140A05FD377AE6
:10060000585A000004E6D6B4460200210116000044
:1006100000742FE5A3E001BD00D85D003D8889C6C8
:100620005436C3174FE4E621DC46349FB0B7F48C50
:100630007B49B03C7EC4755E8EDFCF44B15DDBEAA2
:100640006F4E3A48341F008ECE4DE070AD1A1062E6
:100650005A235C960F0415A51463125D4EB3B21AAB
:10066000F962710D99B9F51AAA88DEEEFC1ACBE091
:100670009ADF69C97CB2193D07ABDA1E4456E1CF57
:100680007A078E44E5A4C11A5B73EA36F9FAC72AE1
:100690009DF9E1EADC63814432809E46E8BAD22AC1
:1006A0005402020A32C2B671AD3C717D7B1F4CDF31
:1006B00092C44DA4FC301AE167065D55FAA90020EA
:1006C000997EB1FD9B8339D5B937EC572BA06804CF
:1006D000CEB76712A95099AE6E6196D580BC3288AC
:1006E000B97E4326570CAFD698D172D6D550DDD7F8
:1006F000116923000062DCEBF7A520F53D0001F451
:1007000001BE0300009221DD8FB1C467FB0200002F
:10071000000004595A504F52514A4D4B4E2A4C2F0B
:1007200030B6B7ABACBBBCA9AABDBECFD0CDCEDB7B
:10073000DCD9DA0D0E0B0F1A05080509050718118B
:10074000130408120C0011241FBECFEFDAE0DEBF45
:10075000CDBF04B603FE18C0809193049091940419
:10076000A0919504B09196048730904BA740B04B70
:1007700059F41092930410929404109295041092DC
:100780009604E0E0F8E3099524E0A0E0B2E001C0BF
:100790001D92A339B207E1F712E0A0E0B1E0ECE36B
:1007A000FBE602C005900D92A030B107D9F70E9478
:1007B00008280C941E3524CC9C01FB019A958115C8
:1007C0009F4120F5832F8170B32FB270AA27732F1A
:1007D00074706627532F5870442734FF0DC08295DC
:1007E000807FAB2B09F08062672B09F08064452B7A
:1007F00009F0806809950895AB2B09F08260672B9A
:1008000009F08460452BB1F38860F4CF80E0F2CF2B
:100810000C9440330895982F92959F7024E0911185
:1008200002C020E0982F892F86958695811511F0BA
:100830002E5F982F892F8695820F08958093360416
:10084000089580933704089521E030E001C0220F1D
:100850008A95EAF780913704822BF3CF21E030E0CC
:10086000A90102C0440F551F8A95E2F7CA0180957D
:10087000909137048923E5CF9B01677091E001C017
:10088000990F6A95EAF763E0369527956A95E1F73F
:10089000B901660F771F260F371FFA01E20FF31F0A
:1008A00040E050E0682F70E08191DF019B01042E51
:1008B00002C0369527950A94E2F7217021952827E2
:1008C000292328272E934F5F5F4F4330510561F74F
:1008D00008959C01A82FA77083E0369527958A95E7
:1008E000E1F7C901880F991F820F931FFB01E80FE1
:1008F000F91F40E050E080E0219130E00A2E02C074
:10090000369527950A94E2F721703327042E01C00B
:10091000220F0A94EAF7822B4F5F5F4F4330510555
:1009200059F70895282F862F903F71F0933068F47F
:10093000253050F4622F70E025E0929F600D711D0C
:10094000112443EB53E098CF08959C5F9230E0F779
:10095000622F70E040EB53E0F6CF903FB9F0933058
:1009600070F4853098F4282F30E063EB73E0A90130
:10097000E5E09E9F400D511D1124CA01AACF9C5F46
:10098000923020F460EB73E090E0F8CF80E00895BF
:100990009091370421E030E0F90101C0EE0F8A9513
:1009A000EAF7D90102C0AA0FBB1F6A95E2F7EA2B4A
:1009B00001C0220F4A95EAF7892F8E23E81303C05E
:1009C000892F822B3ECF2095822F8923FBCF8091C8
:1009D0003F0490913E04981301C008958F5F877083
:1009E000FACF909139048095892380933904282F78
:1009F0002770211110C0891771F09091920492FF15
:100A00000AC086958695869529DF10923904109242
:100A10003B0410923A040895982F909580913404E5
:100A2000892380933404089580913304811531F033
:100A30001092330410923D0410923C040895803EBD
:100A40009105D9F1C8F48133910509F482C048F4C5
:100A50008932910509F472C08A32910509F480C087
:100A6000089589339105E9F082389105D1F08533F5
:100A7000910509F45EC00895843E9105D9F148F4CA
:100A8000823E910539F1833E910549F181EE90E076
:100A90000895863E9105C9F1873E910509F43EC04F
:100AA0000895209191042370211164C02091920433
:100AB00023FF14C089E290E008952091910420FD65
:100AC00045C03091920430FF09C024FD24C083EE5C
:100AD00090E008952091910422FDF7CF0895209190
:100AE000910422FD44C03091920430FD43C024FFA4
:100AF000F5CF11C02091920421FFF0CF8091910495
:100B000084FD09C087EE90E008952091910423FFB1
:100B1000E5CF24FFF7CF80E090E008952091910485
:100B200023FD2BC03091920431FFE1CF84EE90E0A1
:100B300008952091910425FFD1CFBCCF209191043D
:100B400025FD1EC02091920423FFC8CF89E390E0C9
:100B500008952091910426FFC1CF8AE290E0089584
:100B60002091910426FFBACF81E390E0089582EEB0
:100B700090E0089580EE90E0089586EE90E008956C
:100B800085E390E008959091910492FF10C041E0B8
:100B9000282F2471243009F040E031E0282F2871FB
:100BA000283009F030E0431711F02CE0822793FF42
:100BB00010C041E0282F2471243109F040E031E0D9
:100BC000282F2871283109F030E0431711F02CE06C
:100BD00082273091920430FF10C051E0282F2171FC
:100BE000213009F050E041E0282F2871283009F029
:100BF00040E0541711F029E0822731FF10C041E096
:100C0000282F2171213109F040E031E0282F28718F
:100C1000283109F030E0431711F029E0822794FDD4
:100C2000877E08951F93CF93DF9309DFEC01811531
:100C300022E5920708F052C0811540E5940708F0BC
:100C4000CDC0803E910520F58D3C910508F0A1C0F6
:100C5000883A910570F4853A910508F097C0813083
:100C60009105B9F10497813A910598F1C0E0D0E07F
:100C700030C0885A91094B97C8F7C85AD0E0CC0FBA
:100C8000DD1FCD56DE4F0990D881C02DD46421C020
:100C9000811550E49507B0F4C11580E2D80708F03B
:100CA000B3C0C83ED105A8F0CE019A9581159F41E9
:100CB000E8F68D2F68DF182FCE019927C0DEEC01F2
:100CC000D12B07C09927BBDECC27DF70C82BD92BCF
:100CD000D06ACE01DF91CF911F910895803842E50F
:100CE0009407C8F5803652E5950708F05BC0C0341C
:100CF00082E5D807D0F4C03292E5D90708F04BC09E
:100D00008C2F8695869520E2829FC0011124C370A6
:100D100021E030E0A90102C0440F551FCA95E2F757
:100D2000EA01C82BD92BDD68D4CF8C2F8695869508
:100D3000877050E2859FC0011124C37021E030E02C
:100D4000A90102C0440F551FCA95E2F7EA01C82B5A
:100D5000D92BDC68BECF803C52E5950758F48F71E3
:100D6000C03AD245A0F590E0982F8827EC01C46FD7
:100D7000D06AAFCF805C9245809708F077CFDC2FA8
:100D8000CC27CC27DF71C06FD06AA3CFA497D064E3
:100D9000A0CFD0659ECFCF71D0E0DC2FCC27C16F24
:100DA000D06A97CF86958695877020E2829FC00192
:100DB0001124C37021E030E0A90102C0440F551F87
:100DC000CA95E2F7EA01C82BD92BDA6882CFDBDEBD
:100DD000C82FD0E0DC2FCC27D0627BCF8F71D3DE41
:100DE00093E0CC0FDD1F9A95E1F7CC27DF70282F19
:100DF00030E084FF05C050E1859F90011124332726
:100E0000C22BD32BD06965CF8D2F8F71BCDE182FED
:100E1000CE01992714DEEC01D12BDECF80E00895BE
:100E2000F894E82FE295EF70F0E041A18F7021E097
:100E300030E0B90102C0660F771F8A95E2F7CB0157
:100E4000962F9095942391A392A1892B82A37894B5
:100E50000895089508950895982F282F207F203D04
:100E600041F180F4203B31F038F4907E903811F05D
:100E7000203AD1F483E0089581E0203C09F080E03D
:100E8000880F0895203EB1F3203F71F4833F89F02D
:100E900020F4813F71F0823FECCF81E09D3F30F440
:100EA000983F30F4963F21F080E008959E3FE0F3B4
:100EB000089582E00895CF92DF92EF92FF921F9300
:100EC000CF93DF93172FE82FF0E0E851FB4F71111C
:100ED0000CC0E4918E2F7E2F6E2FDF91CF911F914A
:100EE000FF90EF90DF90CF900895E62EF12CC72E63
:100EF000D12CF491EF2F86E0689F90011124CFEF61
:100F0000D0E0C901BE010E941333AB01EE0CFF1CFF
:100F100065E5649FC001659F900D1124E81AF90AE8
:100F20006E2D660F6E0D7E01EC18FD08FE9DD00142
:100F3000FF9DB00D11248B2F169F70011124EF2CF3
:100F4000FF246E01CE18DF087601FE9D6001FF9D33
:100F5000D00C11247E01E61AF108B701169F70012A
:100F6000179FF00C1124EF2CFF24CE19DF09FC9FF2
:100F70007001FD9FF00C11247F2D43305105C1F00D
:100F80002C3F334058F441305105B1F04230510507
:100F900009F0A2CFEB2F8F2D7F2F9ECF443051052C
:100FA00071F04630510509F497CF7B2F8D2D94CFEA
:100FB0007D2DEB2F8F2F90CF7F2FED2D8DCFEF2D10
:100FC0007B2FF8CFCF93982F762F842FC22F692FA6
:100FD00072DF472F282F8C2F90E087D2CF91089572
:100FE00080912A04843028F48370846080932A04DA
:100FF00008958C3AE8F38370886AF8CFCF93DF9333
:1010000080912A0480FD0BC0C0E0D0E020E040E0E9
:1010100060E0CE016AD22196C330D105B9F70E94B3
:10102000A910DF91CF910895FF920F931F93CF9353
:10103000DF93182F062FF42E80912A0480FF0CC016
:10104000C0E0D0E02F2D402F612FCE014ED221964F
:10105000C330D105B9F7D2DFCDB7DEB7E5E00C94E8
:101060008C33CF93DF93EC0120912D049C81892F49
:10107000817090FD822F692F627091FD622F492F40
:10108000447092FD422FD0DF8C8190E001968770F2
:1010900099278C83DF91CF910895982F762F842FF5
:1010A00020912A0420FF07C0692F05DF962F672FA4
:1010B000482F892FB9CF0895CF93DF93EC01EAE24F
:1010C000F4E0438162818C81E8DF8C818F5F8C83C7
:1010D000DF91CF910895CF93DF93EC01EC81F0E0A5
:1010E000ED51FC4F4491EAE2F4E062818181D5DF69
:1010F0008C818F5F8C83DF91CF910895FF920F9346
:101100001F93CF93DF93EC01F12C00E010E08C8172
:10111000980140912D0460912C048F0D53DF0F5FD7
:101120001F4F85E5F80E0330110589F767DF8C81C5
:101130009A8190FF07C08F5F8C83CDB7DEB7E5E063
:101140000C948C338150F8CFEF92FF920F931F9342
:10115000CF93DF93FC018281FF24F39480FF02C0D0
:10116000FF24FA94C0E0D0E020E040E060E0CE014F
:10117000BCD104E010E0E12C809163028E0D84303C
:101180008CF163E00E940633892F082E001C0008B2
:101190008C170D0679F440912D040403A00111244D
:1011A00055954795559547959E0160912C048091E2
:1011B0002B0408DFEF0C01501040F1F62196C330EC
:1011C000D10591F61BDF80916302F1E0FF120EC0A2
:1011D000811591F0815080936302CDB7DEB7E6E0D0
:1011E0000C948B3387FFD1CF8D5FCFCF90E00196EA
:1011F000BE010E942733EFCF82E0EDCFCF93DF9384
:10120000C0E0D0E020E040E060E0CE016ED1219669
:10121000C330D105B9F7C0E0D0E080916202082E5A
:10122000001C0008C817D0055CF180910601082E4B
:10123000001C00088C170D061CF19E0140912D0426
:1012400060912C0480912B04BDDE2196C330D10522
:1012500021F7D4DE8091050190916202980F90935E
:10126000620220910601280F20930601121614F441
:1012700092301CF0819580930501DF91CF91089504
:1012800020E040E060E0CE0130D1DFCFA6E0B0E06A
:10129000ECE4F9E00C946D338D839E83AD81BE81C7
:1012A0001496FC912F2F30E0D9010E940F359B013D
:1012B000AC010E94DD346B017C0180E290E09C0176
:1012C0002F1B3109F901A5E5B0E0A70196010E94A5
:1012D000DD3469837A838B839C839F01DF010E94C5
:1012E00057339B010E945D339B01AC012C0D3D1DCA
:1012F0004E1D5F1D69817A818B819C810E94ED3436
:10130000022F30E00A32A0F5A901440F551F420F09
:10131000531F55954795142F1095E12CF12C85E519
:10132000D82ED01A8D2DE1FC802F9701412F60918E
:101330002C0448DE3FEFE31AF30A83E0E816F104D9
:1013400089F75CDEAD81BE8114969C9181E0911598
:1013500019F0903219F48FEF809304018091040109
:10136000890FED81FE8184832696E8E00C94893311
:1013700085E590E0821B930BAC01440F551F480F8D
:10138000591F57FFC6CF4F5F5F4FC3CF0F931F93B8
:10139000CF93DF938C01C0E0D0E060912C0480916A
:1013A0002B04F8019481209751F4911569F020E005
:1013B00030E040912D0406DEC1E0D0E0EECF9E018A
:1013C00040912D04911511F09E0140E0FBDD219626
:1013D000C330D10511F712DEF801848190E0019647
:1013E000817099278483DF91CF911F910F91089588
:1013F000FB01811520E2920728F4811541E0940752
:1014000038F408959C0130522115304348F0089576
:10141000392F94FF02C03295307F2081232B208307
:1014200099270895462B22FF0FC0982F92959F7001
:101430008F70892B962F92959F706F70692B942FC8
:1014400092959F704F70492B982F9623961309C041
:1014500050E04095509590E04823592381E0452B7A
:1014600009F080E0089590E06115E9F0875B9E4FF8
:10147000FC0180818F3FB1F0E82FE295EF70F0E042
:1014800041A18F7021E030E0B90102C0660F771FE3
:101490008A95E2F7CB01962F9095942391A392A180
:1014A000892B82A308958A5B9E4FE2CF90E061155D
:1014B000A9F0875B9E4FFC0120812F3F91F0E22F26
:1014C000E295EF70E05EF0E0808190E02F7002C066
:1014D000959587952A95E2F7817008958A5B9E4FCE
:1014E000EACF80E00895539A0895FC01EE0FFF1FA4
:1014F000E80FF91FE65BFD4F618340832283089567
:101500000F931F93CF9301E010E0082E01C0000F4E
:101510000A94EAF7C09132049C2F9023911115C0D0
:1015200090913904969596959695891306C01092D8
:10153000390410923B0410923A0486D9C027C09314
:101540003204CF911F910F91089588D9F7CF282F9A
:1015500035EB2303C001112497FF04C08058910983
:10156000892F089580589F4FFBCF8091BB0380FD4A
:1015700014C081FD14C082FD16C08091BA0381158C
:1015800081F08E3180F420E5829FC00111246EE14C
:1015900070E00E942733862F089584E1089588E241
:1015A000089588E0089580E508958091BB0380FD4B
:1015B00017C081FD17C082FD19C08091B903811544
:1015C00099F0883298F428E0829FC001112468E2E3
:1015D00070E00E9427336115710551F0862F089540
:1015E00062E0FCCF64E0FACF61E0F8CF68E0F6CFCC
:1015F00081E008959091170489029001112437FF2A
:1016000003C08093170408952F3731051CF4980FF9
:101610009093170408959C0180E090E0F901E80F91
:10162000F91FE491E41307C091E08927F901E80F5D
:10163000F11D849108950196861780F380E0089546
:10164000E091A603F091A703309739F00190F08163
:10165000E02D309711F00995089580E00895A3E0FA
:10166000B0E0E5E3FBE00C9473339C018091480209
:101670009091490282179307B1F030934902209369
:101680004802E091A603F091A703309761F000842F
:10169000F185E02D309739F083E089833B832A83FD
:1016A000CE01019609952396E2E00C948F33A3E0D6
:1016B000B0E0EDE5FBE00C9473339C0180914602B1
:1016C0009091470282179307B1F03093470220931D
:1016D0004602E091A603F091A703309761F00084E1
:1016E000F185E02D309739F084E089833B832A83AC
:1016F000CE01019609952396E2E00C948F339091E8
:101700002C01913091F0A4E0B2E0EFEF90E02D9148
:10171000821751F0EF3F19F4211101C0E92F9F5FAB
:101720009630A9F7EF3FC9F408959091910497FF7F
:10173000EACFE82FE695E695E695803FA8F7F0E03A
:10174000E65FFD4F877021E030E001C0220F8A95EF
:10175000EAF78281822B828308950E2E000CFF0B04
:10176000EE5FFD4FF8CF90912C01913021F49091D4
:10177000910497FD0CC0E4E0F2E09191891302C05E
:10178000DF011E9252E0EA30F507B9F70895E82F1D
:10179000E695E695E695803FC8F7F0E0E65FFD4FF9
:1017A000877021E030E0A90102C0440F551F8A95DF
:1017B000E2F7CA01809592818923828308958091FE
:1017C0002B0108952FB7F894809142029091430223
:1017D000A0914402B09145022FBF0895CF93DF93AB
:1017E000C091340480913804C82B80913304811552
:1017F000F1F0E8DF20913C0430913D04821B930B13
:101800008838934108F010D9D091330480912C018D
:10181000813021F48091910487FD0DC086E024E0A1
:1018200032E090E0815058F49111FED8CD2B8C2FEE
:10183000DF91CF9108958EE12CE032E0F2CFF901F3
:1018400041919F01411571F39F5FECCF962F20913D
:10185000920422FF0FC0682F660F660F660F692B78
:10186000609339040E942404ADDF90933B0480937D
:101870003A0408950C94240490913304292F2823CA
:10188000211559F08095892380933304811531F017
:1018900099DF80933C0490933D04089580E090E0AC
:1018A000F8CF90DF2091BE033091BF03232B211589
:1018B00021F080938602909387022091C00330919B
:1018C000C103232B211521F080938402909385027C
:1018D000E091A603F091A703309759F00680F781B5
:1018E000E02D309731F082E08093BC038CEB93E0E5
:1018F00009950895611509F441C0E3E3E80FE33168
:1019000048F4F0E0E05EFA4C0C943A332EDE819518
:101910008093BF03C6CF29DEFBCF27DE819580935E
:10192000BE03F8CF22DEFBCF40DE8093C003F2CFB0
:101930003CDE8195FACF39DE81958093C103EACFF1
:1019400034DEFBCF815D990B21E030E001C0220F36
:101950008A95EAF78091BD03822B8093BD03DACF8D
:101960008091BB0381608093BB03D4CF8091BB0384
:101970008260F9CF8091BB038460F5CF4091BE03B4
:101980008D3C59F48091BF0387FF0DC01092BF03B7
:10199000411559F41092BA0308C08E3C81F480912D
:1019A000BF0318169CF3411581F08091C0039091FC
:1019B000C103892B8111AECF1092B903ABCF8F3CFD
:1019C00041F447FFF0CF1092BE038091BF03811511
:1019D000E0CF803D19F41416B4F3E5CF9091C00325
:1019E000893D29F41916FCF61092C003DCCF8A3D1C
:1019F00019F497FFD8CFF8CF9091C1038B3D29F40C
:101A000097FFD1CF1092C103CECF8C3D19F4191698
:101A1000CCF3C9CF9FE2980F983090F4815D990B79
:101A200021E030E0B90102C0660F771F8A95E2F726
:101A3000CB0180959091BD0389238093BD03B3CFE3
:101A40008D3D31F48091BB038E7F8093BB03ABCF80
:101A50008E3D21F48091BB038D7FF7CF8F3D09F040
:101A6000A2CF8091BB038B7FF0CF2FB7F89460910A
:101A700042027091430280914402909145022FBF2F
:101A80000895FC019B0180913802909139028617DC
:101A9000970740F0672B29F48091E8008E778093B8
:101AA000E800C90140E0009741F4411106C080916F
:101AB000E80082FF2FC080E0089520917F03211568
:101AC000A9F12530A9F12091E80023FD2DC0209136
:101AD000E80022FDECCF2091E80020FFE4CF309118
:101AE000F3002091F200009719F02830310558F0EA
:101AF00041E02830310509F040E02091E8002E77E0
:101B00002093E800D0CF41914093F10001972F5FDF
:101B10003F4FE9CF80917F03811541F0853041F03F
:101B20008091E80083FFC3CF81E0089582E00895AB
:101B300083E008958091320287FF13C08091E8000E
:101B400082FF06C08091E8008B778093E8000895BB
:101B500080917F038111F2CF089580917F038115D9
:101B6000D9F38091E80080FFF8CF8091E8008E776C
:101B7000ECCF2091E4003091E50095E6A901209199
:101B8000EC00822F817020FF06C08091E80080FF6A
:101B900006C080E008952091E80022FD1AC08091DF
:101BA0007F03811589F0853089F08091EB0085FDF8
:101BB0000FC02091E4003091E50042175307F9F27D
:101BC0009A95E1F684E0089582E0089583E008950F
:101BD00081E00895E8EDF0E080818E7F80831092AF
:101BE000E2001092DA001092E100A0EEB0E08C91D9
:101BF00081608C9380818F77808319BCA7EDB0E0E2
:101C00008C918E7F8C9380818F7E808310923102A5
:101C10000895EF92FF920F931F93CF937C018B0156
:101C2000A8DFC82F811116C08091E80085FD0AC089
:101C30008091E8008E778093E8009BDF8115A1F307
:101C4000C82F08C0F70181917F018093F1000150F6
:101C5000104051F78C2FCF911F910F91FF90EF9073
:101C60000895A4E0B0E0E7E3FEE00C946E337B015E
:101C7000142FD22E4A832B830C83842FEDD881110D
:101C80003AC082E0E816F10489F083E0E816F10436
:101C900041F081E0E816F10451F12496E7E00C945C
:101CA0008A3317E0073F31F014E004C087EF16E0F5
:101CB000D812FACF198380917F03843071F7809115
:101CC0001F018F708093E90040E050E064E070E015
:101CD000CE0101969EDF8111E0CF8091E80085FD65
:101CE000DCCF8091E8008E778093E800D6CF173F55
:101CF000D9F615E0DFCF12951F70DCCFEF92FF927F
:101D00000F931F93CF937C018B0133DFC82F811179
:101D100016C08091E80085FD0AC08091E8008B77AD
:101D20008093E80026DF8115A1F3C82F08C08091B9
:101D3000F100F70181937F010150104051F78C2F82
:101D4000CF911F910F91FF90EF900895A7E0B0E021
:101D5000ECEAFEE00C9470338C0108511F4F809127
:101D60007F03843009F062C0809124018F708093DA
:101D7000E9008091E80082FF59C08091E80085FF6A
:101D800055C040E050E064E070E0CE010196B6DF5F
:101D90008091E80085FD05C08091E8008B778093F5
:101DA000E800FA808F2D58D8282FFD828B818E83F2
:101DB0008C818F83211108C0E981E450E43078F6EA
:101DC000F0E0E958FE4F208130E0321740F6FE0186
:101DD0003596E30FF11DF0804FB7F894D8011196B6
:101DE000EC911197F0E0CF01019612966C9170E0A2
:101DF0000E942733D8015C915817190619F44FBF78
:101E00003F5FE3CF13968D919C911497E80FF91FD4
:101E1000F08211968C91119790E0019612966C9138
:101E200070E00E942733F8018183E9CF2796E5E02F
:101E30000C948C33E091A603F091A703309739F00E
:101E40000284F385E02D309711F060E20995089542
:101E5000A3E0B0E0EEE2FFE00C946D337C01162FBE
:101E6000D42EC22E8091AD02843069F5E091A20299
:101E7000F091A3023097B9F1970121503109C901BE
:101E800063E070E00E941333B901681B790B19837A
:101E90004A83CB824E2D461B9E012F5F3F4F88E821
:101EA00092E00995E091A602F091A702309739F0EF
:101EB0000C2D2D2D412FB70188E892E0099523962E
:101EC000E8E00C94893382E0E816F10409F454C088
:101ED00083E0E816F104A9F081E0E816F10409F4C2
:101EE0007AC0E12CF12CE091A402F091A502309788
:101EF000C9F20C2D2D2D412FB70188E892E00995EC
:101F0000D1CF862F807F803B19F188F4803929F169
:101F1000803A41F1E0918E02F0918F02803819F7FA
:101F2000309709F32C2D4D2D612F6F700DC0803E21
:101F3000F1F0803FC1F6623FB1F6E0919402F0917A
:101F4000950262EF309779F288E892E00995AACF7E
:101F5000E0918A02F0918B02E3CFE0918C02F09144
:101F60008D02DECFE0919002F0919102D9CFE09105
:101F70009202F0919302D4CF862F807F803D81F032
:101F8000803F99F0E0919602F0919702803C09F031
:101F9000AACF309709F4A7CF4D2D612F6F7017C0CE
:101FA000E0919802F0919902F4CFE0919A02F091B9
:101FB0009B02633F39F0613F09F095CFE0919C02AD
:101FC000F0919D024D2D612F309709F48CCF88E858
:101FD00092E0099567CFE0919E02F0919F02683FE1
:101FE00038F4663F09F07FCFE091A002F091A102A2
:101FF000309709F478CF612F88E892E0099552CFA5
:10200000982F9093E900891771F07091EC0020915E
:10201000ED005091F00021FD09C09F5F973089F7D6
:102020008093E9000895762F242F50E03091EB0043
:102030003E7F3093EB003091ED003D7F3093ED001B
:102040003091EB0031603093EB007093EC00209303
:10205000ED005093F0002091EE0027FDDECF0895B3
:10206000A0E0B0E0E6E3F0E10C946D33C8EDD0E021
:1020700088818F7E8883E7EDF0E0808181608083B6
:1020800084E082BF81E08093310288818E7F8883E3
:1020900002EE10E0F80110821092DA0081EEC82EF4
:1020A000D12CF601108288818F778883888180689F
:1020B000888388818F7D888319BC10927F0310925A
:1020C00030021092690210922F0290EEE92EF12C4C
:1020D000F70180818B7F808388818160888342E0E3
:1020E00060E080E08DDFF60180818E7F8083F801E3
:1020F000808181608083808188608083F701808116
:102100008E7F8083888180618883CDB7DEB7E8E0E9
:102110000C948933E0913F0490913E0429E0E91347
:1021200002C080E00895AE2FB0E02E9FF001112490
:10213000E05CFB4F3181361306C03081381303C099
:102140003581341304C0FD013196E770E8CF81E09A
:1021500008953BB1377F2BB128604FB7F8948AE4DC
:1021600092E0FC010196508168E02BB9000000C0AC
:1021700057FF3BB9550F000000C000C000C03BB97D
:1021800000C06A9591F752E08335950751F74FBF2C
:102190008FE594E00197F1F700C00000089581E019
:1021A0008093E00080E28093D8001092C9008FE114
:1021B0009EE40197F1F700C0000087E090EBDC019E
:1021C0008093930490939404A0939504B093960401
:1021D00088E19CE00FB6F894A895809360000FBE4C
:1021E00090936000FFCF282FCB01BA0130917F037D
:1021F0003430C9F42093E9002FEF3091E80035FD29
:1022000006C035ED3A95F1F700002A95B1F7209117
:10221000E80025FF08C040E050E0FBDC8091E800CA
:102220008E778093E8000895792F603229F440E298
:1022300050E0682F82E0D7CF0895CF93DF93D82F57
:10224000C92F48E050E0682F792F81E0CCDF88E08B
:10225000ED2FFC2FAAE3B2E001900D928A95E1F7F1
:10226000DF91CF910895BC0140E250E084E0BBCF04
:10227000BC0146E050E084E0B6CFBC0143E050E052
:1022800084E0B1CF9091920492FB222720F9281785
:1022900079F080FB92F9909392046091910470918F
:1022A000920484E090E00E94A63482E00C94F10451
:1022B00008951F93CF93DF93962F122F632F8330B0
:1022C000D8F49330C8F44530B8F4C42FD0E0CC0F24
:1022D000DD1F2AE0929FC00DD11D11249EE1899F30
:1022E000C00DD11D1124CE0189960E948C34612F1E
:1022F000CE018A960E948C34DF91CF911F91089570
:102300000F931F93CF93DF93C62F142F022F632FAA
:10231000833010F5C33000F524E0C29FE0011124A2
:102320003CE0839FC00DD11D1124CD57DF4F81E0CC
:1023300084279E01280F311D280F311DC9010E94DD
:102340008C3481E090E0111102C083E090E0602FB6
:102350008C0F9D1F0E948C34DF91CF911F910F91A4
:10236000089580912C01813061F58091910487FF5F
:1023700028C034DA80930B0240E250E066E873E054
:102380008AE092E00E944734892BD1F080E2EAE0B3
:10239000F2E0A6E8B3E001900D928A95E1F7E091B2
:1023A000A603F091A703309759F00480F581E02D42
:1023B000309731F086E080930A028AE092E0099536
:1023C00008950CDA8093020248E050E068EA73E076
:1023D00082E092E00E944734892B91F388E0E2E0AA
:1023E000F2E0A8EAB3E001900D928A95E1F7E0915E
:1023F000A603F091A703309719F30280F381E02D33
:102400003097F1F282E092E0DACFCF93C82F8115B6
:10241000A1F08238A1F414D981FD0FC089E36FD9EE
:10242000A0DF2FEF37EE83E0215030408040E1F70E
:1024300000C0000089E397D994DFCF9108958338D5
:1024400089F4FED880FDF9CF83E559D98ADF9FEF63
:1024500021EE34E0915020403040E1F700C0000010
:1024600083E5E9CF843889F4EBD882FDE6CF87E4B1
:1024700046D977DF8FEF91EE24E0815090402040E5
:10248000E1F700C0000087E4D6CF8CEF8C0F813AD3
:1024900078F580912C01813069F0E4E0F2E08AE087
:1024A00092E02191C21701F18E179F07D1F78C2F6F
:1024B00026D9C2CF8091910487FFEFCFEC2FE6950C
:1024C000E695E695F0E0E65FFD4F828190E04C2FC7
:1024D000477021E030E002C0220F331F4A95E2F737
:1024E00082239323892B19F38C2F3DD93ADFDFCF39
:1024F00080E28C0F883068F4C77081E090E001C002
:10250000880FCA95EAF7C0913404C82BC0933404ED
:1025100093CF8BE58C0F833030F42C2F2452330B68
:10252000C9019DD88ACFE8E5EC0FEB3148F4F0E023
:10253000EE0FFF1FE753FE4F80819181B8D87DCF0A
:1025400083E38C0F833108F078CF61E08C2FD2D9F0
:1025500074CF811509F445C0823849F471D881FFE0
:1025600040C089E3CCD8FDDE89E3FDD8FACE8338BC
:1025700041F466D880FF35C083E5C1D8F2DE83E53B
:10258000F4CF843841F45CD882FF2BC087E4B7D8FD
:10259000E8DE87E4EACF9CEF980F913A30F390E2BF
:1025A000980F983050F4877091E001C0990F8A9588
:1025B000EAF7892F0E940C05D9CF9BE5980F93303D
:1025C00018F480E090E04BC898E5980F9B3118F420
:1025D00080E090E06CC893E3980F933110F460E0D2
:1025E00089C908951F93CF93DF93182FEB010DDF57
:1025F000209731F4812FADDFDF91CF911F910895A6
:102600008FE99FE00197F1F700C000002197F0CF1C
:10261000811531F090913404892B80933404A1CE3C
:102620000895811519F00E940C059BCE0895EF9234
:10263000FF920F931F93CF93DF93C62FD42F122FA8
:10264000811599F060932604BDD890932E02809353
:102650002D02C77081E001C0880FCA95EAF7D8DF64
:10266000CDB7DEB7E6E00C948B3380912604681377
:102670002FC0E0902D02F0902E02A4D88E199F0951
:10268000883C910528F500E20D0FCD1799F0C77031
:10269000FF24F3948F2D01C0880FCA95EAF7C1DF9C
:1026A000083040F48D2F877001C0FF0C8A95EAF73F
:1026B0008F2DAEDF60E070E0812F94DF083080F670
:1026C000D77081E001C0880FDA95EAF7AADFC8CF9A
:1026D000C77081E001C0880FCA95EAF7F7CF81156E
:1026E00031F090913804892B809338043ACE0895C4
:1026F000811539F0809590913804892380933804AE
:1027000030CE089580912204811521F082E2F0DF1D
:102710001092220408951092340480912C0181308B
:1027200021F58091910487FF20C0ECE0F2E08EE17A
:10273000DF011D928A95E9F780E090E00E942F0B5F
:1027400080E090E00E94570B109238040ADE86E089
:10275000ECEBF3E0DF011D928A95E9F71092BA03E2
:102760001092B9031092BB039CC8E4E0F2E086E04B
:10277000DFCFD1DF2FEF84E39CE0215080409040F9
:10278000E1F700C0000088E19CE00FB6F894A8953E
:10279000809360000FBE90936000FFCFAAE2B0E08C
:1027A000E4EDF3E10C94723382E392E0FC010196D4
:1027B0002091F100208322E08A339207B9F78091BB
:1027C0003302893009F457C0C8F4823009F4B2C02A
:1027D000833009F482C0813081F18091E80083FF69
:1027E000E6C080913202909133029A3008F0DFC047
:1027F000E92FF0E0ED5CFA4C0C943A338A3009F49E
:1028000089C08B3051F780913202813231F780914B
:10281000360290913702892B01F78091E800877F7B
:102820008093E80087D981E090913402911101C032
:1028300080E080932C016FDFD0CF80913202813A0B
:1028400061F68091E800877F8093E80080913602EE
:1028500090913702892B59F060E080E090E070E0C1
:1028600010D98091E8008B778093E800B6CF68E0BC
:102870008AE392E0F4CF80913202813209F0ADCF49
:1028800080913602909137028D7F892B09F0A5CF78
:102890008091E800877F8093E8008091E80082FFC4
:1028A00017C09091F3008091F200029731F480916B
:1028B000F100813011F0863021F48091F100809395
:1028C0002B018091E8008B778093E80033D985CF86
:1028D00080917F038111E1CF80CF80913202813AD4
:1028E00009F07BCF8091360290913702892B09F055
:1028F00074CF8091E800877F8093E8008091E800A2
:1029000080FFFCCF80912C018093F1008091E80042
:102910008E77DACF80913202813209F05ECF8091DA
:10292000E800877F8093E80005D980913502809385
:102930002A0153CF80913202813A09F04ECF809123
:10294000E800877F8093E8008091E80080FFFCCF5B
:1029500080912A01D9CF803889F0823841F5809161
:1029600036028F70873018F58093E9008091EB0074
:1029700085FB882780F91092E90006C080916902E2
:10298000880F90912F02892B9091E800977F909368
:10299000E8008093F1001092F1008091E8008E77BA
:1029A00023C0811116C080913402813009F18091D9
:1029B000E80083FF0AC08091E800877F8093E800E9
:1029C0008091EB0080628093EB00AA96E3E00C9488
:1029D0008E33823061F780913402811581F010923C
:1029E000E9008091E800877F8093E800A3D8DFCFDB
:1029F00081E0933009F080E080936902F0CF80910C
:102A000036028F702FEF280F263088F68093E9006A
:102A10002091EB0020FFE3CF933031F48091EB0065
:102A200080628093EB00DBCF9091EB0090619093FC
:102A3000EB0021E030E0A90102C0440F551F8A9548
:102A4000E2F74093EA001092EA008091EB00886080
:102A5000E8CF8111ACCF109134021F778091E30051
:102A60008078812B8093E3008091E800877F8093BA
:102A7000E80060D88091E80080FFFCCF8091E300FF
:102A800080688093E30083E0111101C082E08093AD
:102A90007F038DCF8058823008F089CF8091340237
:102AA000909135028C3D53E0950799F583E08A8338
:102AB0008AE289834FB7F894DE01139620E03EE066
:102AC00051E2E32FF0E050935700849120FF03C0C0
:102AD00082958F703F5F8F708A30C8F0895C90E07C
:102AE0008D939D932F5F243161F74FBF8091E80054
:102AF000877F8093E8006AE270E0CE0101960E9431
:102B0000410D8091E8008B778093E80050CF805D85
:102B1000E6CF292F33272330310509F44EC078F54D
:102B20002130310509F488C08FEB90E0E8E7F2E04E
:102B30002230310509F03BCF2091E800277F209318
:102B4000E80020913802309139028217930708F487
:102B50009C0140E02115310509F073C0411171C09D
:102B60008091E80082FDCDCF80917F03811549F2ED
:102B7000853039F28091E80083FFF2CFC2CF809197
:102B80003602909137022132310509F446C02232D3
:102B9000310509F00CCF8330910508F008CFFC0116
:102BA000EE0FFF1FE65CFE4F0190F081E02D895C87
:102BB0009E4FDC018C9190E010C09C013327823045
:102BC00021F12330310568F4232BB9F4EBE8F3E06D
:102BD000E4918E2F90E0EBE8F3E0009709F4E7CE64
:102BE000ABCF2330310509F0E2CEE9E4F3E0E49124
:102BF0008E2F90E0E9E4F3E0F0CFE3E7F3E0E49137
:102C00008E2F90E0E3E7F3E0E8CFE7E6F3E0E4912E
:102C10008E2F90E0E7E6F3E0E0CF8330910508F0F7
:102C2000C6CEFC01EE0FFF1FE05CFE4F0190F0816D
:102C3000E02D89E090E080CF82E190E0E7E3F3E0EF
:102C40007BCF80917F03811509F45BCF853009F438
:102C500058CF8091E80083FD54CF8091E80082FD39
:102C60007FCF8091E80080FF75CF9091F300809135
:102C7000F2002115310519F08830910550F041E03E
:102C8000089709F040E08091E8008E778093E80093
:102C900061CF44914093F100319621503109019662
:102CA000E8CF803809F083CE8091E800877F809359
:102CB000E800809130028093F1006FCE811177CED1
:102CC00010913402123008F072CE8091E800877FB4
:102CD0008093E800109330020E949A0D111519F1AB
:102CE00084E080937F0342E061EC81E089D942E295
:102CF00061EC84E085D942E261EC82E081D942E274
:102D000060EC83E07DD942E361E885E079D942E374
:102D100060E886E075D980917F03843051F482E0C9
:102D200080932D0144CE8091E30087FDD9CF81E0CF
:102D3000D8CF81E0F5CF0F931F93CF93DF938330EC
:102D400030F5633020F5453010F5C42FD0E0CC0FBE
:102D5000DD1F2AE0629FC00DD11D11243EE1839F3B
:102D6000C00DD11D1124CE0189960E946B34082F0D
:102D700010E0102F0027CE018A960E946B34980134
:102D8000282BC901DF91CF911F910F91089580E009
:102D900090E0F8CFFF920F931F93CF93DF93F42E21
:102DA000833068F5633058F524E0629FE001112418
:102DB0003CE0839FC00DD11D1124CD57DF4F81E032
:102DC00084279E01280F311D280F311DC9010E9443
:102DD0006B34082F10E0102F002781E090E0F110F5
:102DE00002C083E090E08C0F9D1F0E946B3498011D
:102DF000282BC901CDB7DEB7E5E00C948C3380E019
:102E000090E0F8CF2091820330918303232BC9F403
:102E1000703F39F4603FA9F4809180039091810361
:102E20000895733038F4653060F4833050F4462FE1
:102E3000672F81CF7D3F41F4633018F441E0833048
:102E400050F080E090E008957C3FD9F76330C8F7F8
:102E50008330B8F740E09ECFA0E0B0E0E2E3F7E1D6
:102E60000C946E337C010091370480913604082B5A
:102E7000C2E0D0E010E0C8010C2E02C09595879505
:102E80000A94E2F780FD09C02197A8F7D12C8D2D77
:102E9000CDB7DEB7E7E00C948A33DC2EB7018C2F78
:102EA000B1DF0E941206019779F3F1CF0F931F93C0
:102EB000CF93FC0187819085009789F485810081FB
:102EC0001181811581F0611571F0C801C5DFC82F2E
:102ED000682FC8010E949204B8018C2F93DFCF9114
:102EE0001F910F910895C8010E94AD04C82FF4CF1F
:102EF000CF93DF93D82FC92FAFDF6D2F7C2F82DFC9
:102F00000E941206DF91CF910895FC018481811502
:102F1000B1F0878190850097A1F00E941206282FBA
:102F200092959F709630B9F080F4925F9F709230C6
:102F300030F4203FD1F058F481E0283E58F080E092
:102F4000089580819181D4DFEACF9A5FEFCF81E04D
:102F5000243FA9F7089591E0813F09F090E081E0D6
:102F6000283E08F080E0892B089581E00895382FED
:102F7000292FCB01A32FB22F893223E09207A1057D
:102F8000B10520F489529F4F0C946B3480E0089572
:102F900085E290E00E946B348A3589F486E290E005
:102FA0000E946B348C3959F487E290E00E946B34B4
:102FB00091E0853609F090E0892F8170089580E0D6
:102FC000FCCFA0E0B0E0E7EEF7E10C946C33EC014D
:102FD0008881811509F1813009F045C089818130EE
:102FE00051F48A81239660E570E0893311F060E046
:102FF00070E0F8DAEDCF823021F48A81239605DA89
:10300000E7CF833021F48A812396A3DAE1CF84309D
:1030100041F022968111DCCFCDB7DEB7E9E00C9408
:1030200088338A81239620E030E09AE0682F60534D
:10303000770BAB016A30710560F02115310551F352
:10304000EFE9FFE03197F1F700C0000021503109AE
:10305000F4CF929FB001939F700D11249A01260F17
:10306000371F8991E3CFE82FF0E0E850FE4FB4908E
:10307000282F26952695269530E0F901E851FE4F38
:10308000E4908770F12C082E02C0F594E7940A941E
:10309000E2F7E0FAEE24FF24E0F8F901E852FE4FEF
:1030A000C490D12C082E02C0D594C7940A94E2F79C
:1030B000C0FACC24DD24C0F8F901E853FE4F049196
:1030C00010E002C0159507958A95E2F70170112767
:1030D000E114F10411F081EE98D9C114D10411F07A
:1030E00086EE93D960E070E08B2D7CDAC114D104B8
:1030F00011F086EE2EDAE114F10411F081EE29DAF6
:103100000115110521F060E070E08CE26BDA219688
:103110005FCFA6E0B0E0EFE8F8E10C946E330CEC82
:1031200013E087EAE82EF12C98E0D92E46E050E033
:10313000B701CE0101960E945B34F8018D2D1192EA
:103140008A95E9F7B8016C5F7F4F89819A810E9467
:10315000F809F80191838083B8016B5F7F4F8B8101
:103160009C810E94F809F801938382838D81868374
:103170008E818783F6E0EF0EF11C085F1F4F87ED0D
:10318000E816F10499F62696E7E00C948A33A6E057
:10319000B0E0EDECF8E10C94663380907D03909004
:1031A0007E0381E090E090937E0380937D033BEC6F
:1031B000A32E33E0B32EC12CD12C10E0360100E059
:1031C00019C021E030E0123021F0F701859195918E
:1031D0009C01452D602F812F6CD8539422E0E20E84
:1031E000F11C35E05312EDCF0F5F85E0680E711CC6
:1031F000033049F0C301880F991FDC01A157BC4F70
:103200007D01512CDECF750100E021E030E012306D
:1032100021F0F701859195919C0141E0602F812F6C
:103220006FD821E030E0123029F0F7013296859115
:1032300095919C0140E0602F812F62D80F5FB4E030
:10324000EB0EF11C033009F71F5F2CE0A20EB11C3E
:103250003FE0C30ED11C133009F0B0CFFE01319610
:1032600086E0DF011D928A95E9F707EA10E07F0109
:1032700046E050E0B801C7010E94AA340A5F1F4F20
:10328000073D1105A9F790927E0380927D03269653
:10329000EFE00C948233A0E0B0E0E1E5F9E10C94BA
:1032A0006733FC018280648081E08483E3EEF3E095
:1032B0009490E2E6F4E0E49100912D040695015823
:1032C00010E0000F111F012F1127C3E5D2E0C12C20
:1032D000D12CAA24AA94B12C77247A94E919EE2E41
:1032E000F12C83E0881630F480912B048883809140
:1032F0002C048983611017C01B821A8296014A81AF
:10330000698188810E94E2078FEFC81AD80A259642
:1033100083E0C816D10429F70E94FE07CDB7DEB7B7
:10332000EEE00C9483338B818115E9F081508B831F
:10333000789EC00111246C8170E00E941333FB0160
:10334000FF27ED51FC4F8491E82FE9197E9EC001C3
:103350001124B7010E94133380912D04689FB0019E
:1033600011247A83CBCF0E942334B5010E942733E6
:10337000801791071CF683E0881688F00E9423349A
:10338000B5010E94273388830E94233420912C04A6
:103390002695622F70E00E942733280F29831A8216
:1033A00080912D04893C20F088EC8C838B83A6CF00
:1033B0008431D8F784E1F9CF0F93CF93DF93CAE23A
:1033C000D4E0488159816A817B8188E090E00E9445
:1033D0009E34288139814A815B816C817D818E8117
:1033E0009F8100E20E94B533622F83E290E00E9449
:1033F0008C34DF91CF910F910895EAE2F4E085E0FB
:10340000808311828FEF828383831482CF01D4CF94
:1034100080912E04833018F48F5F80932E048AE20B
:1034200094E0CACF80912E04811519F081508093C9
:103430002E048AE294E0C0CFA0E0B0E0E2E2FAE13C
:103440000C946833182FF62E042FE22E90912A0444
:1034500090FF23C0E92FE695E695AE2FB0E0A45B80
:10346000BE4F8C91809328049C7F9430D9F4612FB7
:103470007F2D842F0E945B07962F672F482F892F5F
:103480000E94140810932B04F0922C0400932D0436
:10349000E11419F08AE294E08FDFCDB7DEB7EDE0FA
:1034A0000C948433823019F400912D04EBCF8630D4
:1034B00019F410912B04E6CF8930D9F3893111F733
:1034C000E9518E2F8170782EE695F0E0ED51FB4F9B
:1034D000E491CE2FD0E0A12CB12CC12CD12C83E0D3
:1034E000882E912CC501B4010E941333812F7110D5
:1034F00012C0860F9601402F6F2D0E94E2078FEFBA
:10350000C81AD80AAC0EBD1E83E0C816D10451F704
:103510000E94FE07B7CF861BEDCFEAE2F4E081817F
:1035200021E043816281885F87CFEAE2F4E0818114
:1035300021E04381628188507FCFEAE2F4E062813A
:1035400021E1620F08F46FEF21E04381818174CFA4
:10355000EAE2F4E0628121E1621B08F460E021E02C
:103560004381818169CFEAE2F4E0438121E1420FA6
:1035700008F44FEF21E0628181815ECFEAE2F4E05E
:10358000438121E1421B08F440E021E06281818116
:1035900053CF90912A0490FF2CC0811559F18B32A2
:1035A00058F58F73880F880F90912A049370892B98
:1035B00080932A04611519F08AE294E0FDDE60919F
:1035C0002A046695669570E04BE050E087E091E054
:1035D0000E943A34892B91F01092290481E0809363
:1035E000710220E040912D0460912C0480912B0405
:1035F00023CF089581E0D6CF8AE2D4CF81E08093B3
:1036000029040E94E20B90936F0280936E02E6CF32
:1036100080912A04869586958F5F8B3208F081E031
:1036200061E0B7CF80912A04869586958A9509F442
:103630008AE261E0AECFA9E0B0E0E1E2FBE10C9408
:1036400063338C01DC0114968C91811509F4C2C09E
:1036500061E0C8012BDC7C0180912104811136C01E
:10366000F8018581811509F469C0E114F0E5FF06D0
:1036700008F04EC0E11420E2F20608F0AFC0E114F9
:1036800037E0F30619F1F0F4C701805E910908975D
:10369000E8F030913404809138042091330499E0AB
:1036A000F801ADE0B4E001900D929A95E1F7F09247
:1036B0001504E092140410921704832B822B80933C
:1036C0000C0404C0E1145FE0F50619F7D801159663
:1036D0004C91411185C123E7E2162CE7F20609F46B
:1036E00069C0A2EAEA16A2E5FA0609F491C208F056
:1036F00066C2C70190528115904208F47BC2B1EEB8
:10370000EB16F10409F484C2E5EEEE16F1045BC297
:1037100090EEE91692E5F90650F4A0E6EA16A2E565
:10372000FA06A0F6C701925580349105B1CF9701F2
:1037300027573C472530310508F0ABCFF9E7EF16A6
:10374000FCE7FF0609F04EC02091140430911504E7
:10375000232B81F18115A1F081E00E94FA0A80916A
:103760000C040E946F1389E0EDE0F4E0A3ECB3E0F9
:1037700001900D928A95E1F7809117048093C2031E
:1037800086E0F801A3ECB3E001900D928A95E1F791
:103790008091C2038093210483EC93E04CDF10926C
:1037A0002104D80115968C91811104C080910C04DC
:1037B0000E947813809139048770811559F0F801BF
:1037C0008581811539F08091920482FF03C082E0E7
:1037D0000E94F1042996E2E10C947F33F80186817E
:1037E000803156CFBAE7EB16BCE7FB0609F06ECF87
:1037F000811509F4CAC0A0901404B0901504E0919A
:103800000C04E887E983BE016F5F7F4FC5010E940A
:10381000F8092C01F981F987FCECCF2EF3E0DF2EBB
:10382000EE24E394F12C22242A94D60117963C909E
:10383000179733FE54C06D907C90119712968D901F
:103840009C90139746145704B9F41496BC91BF8307
:10385000232DF60146816B2F89850E94120A81155E
:1038600059F08F810E940804281634F4D601159669
:103870009C917401F92A282E48145904C9F431FE88
:1038800017C0F601F581FF83232DD60116964C91C2
:103890006F2F89850E94120A811551F08F810E9435
:1038A000080428162CF4F60194817301F92A282EB5
:1038B00030FE15C0FFEF2F1212C021E0E216F10416
:1038C00071F4232DD60116964C9160E089850E94F3
:1038D000120A811521F0F60185817401F82AF8E0B9
:1038E000CF0ED11C2CE034E02C153D0509F09DCF06
:1038F00031E0E316F104F1F5988592959F704885C3
:10390000942B9F7081E0403108F480E0F82EF2940F
:10391000E0EFFE22F92AA11450E2B50620F5A11429
:1039200081E0B80608F055C0EA2C8F2D8D704A2D25
:10393000811509F451C06AE08BE397E00E940B0BFC
:10394000282F30E02115310551F44E2D6EE185E12F
:1039500097E00E940B0B282F30E0811549F0F90108
:10396000FF297F0107C0C50190528115904390F156
:10397000E12CF12C87E0E8E1F4E0DF011D928A956B
:10398000E9F7F0922004E0921F0480911F049091C7
:103990002004892B09F40ECFF8018581811539F0B7
:1039A0008FEF0E94FA0A809117048093160486E034
:1039B000F801A8E1B4E001900D928A95E1F78091B9
:1039C00016048093210488E194E035DE10922104EE
:1039D000F1CEFB28BB24A8CF68E083E397E0AECF0D
:1039E000C70197578038910508F0EFC6BE2CF0E16B
:1039F000EF1608F0DFCE68E273E080E090E0B7DA1F
:103A00008111D8CEC12CD12C7601B11042C074E006
:103A1000272EAE014F5F5F4F5E834D83AD81BE8128
:103A2000E22D1D92EA95E9F746015701FFEF8F1A43
:103A30009F0AAF0ABF0AC701B60199DA89838115C7
:103A400009F4B8CE813009F0A6C02601370122E082
:103A5000420E511C611C711CC501B40188DA382E5C
:103A60008A83811509F4A6CE8FEF830D833028F564
:103A7000C301B2017CDA8B83811519F0CE01019666
:103A8000A0DA4601570133E0830E911CA11CB11C42
:103A90004BC029E2C21623E0D206E104F10409F486
:103AA00089CEC701B60163DA3FEFC31AD30AE30A2E
:103AB000F30A8111EECFBA94A8CF8BEF830D833038
:103AC000B0F54601570143E0840E911CA11CB11CC6
:103AD000C301B2014CDA8B83811531F1C501B40108
:103AE00046DA8C838115C9F0AB80BC8051E0A51605
:103AF0005FEFB50610F0BA2CAA2486E0381651F014
:103B000097E0391619F0C5010E945226C5010E949E
:103B1000842603C0C5010E9452264601570154E085
:103B2000850E911CA11CB11C7501640177CFA4E026
:103B3000530142013A12F8CFC301B20118DA782ECC
:103B400046015701B4E08B0E911CA11CB11CC701AA
:103B5000B6016D5F7F4F8F4F9F4F09DA711409F4E3
:103B600029CE811509F426CE8150990B4FEF489F3D
:103B70009001499F300D1124E72DE150FF0B2E0FCE
:103B80003F1F2150310980F28FE99FE00197F1F743
:103B900000C00000F6CFCE01019613DAC5CF109217
:103BA00034040E9414050E94E20B88579C4E9093A7
:103BB00024048093230481E080932204FBCDF2EB64
:103BC000EF16F2E5FF06E9F525EE30E02770332722
:103BD00081E090E001C0880F2A95EAF72091250442
:103BE000309122043115E1F04115A9F0282B2093E2
:103BF0002504E0CDD80116968C91803110F58F2DDB
:103C000099278F7199278230910511F04297DBCF68
:103C100021EE30E0DBCF8095822380932504CACD4E
:103C2000322F3823311569F0982F90959223909375
:103C300025040E940C05D80115968C91811509F474
:103C4000B9CD80912204811509F4D1C0C09034040B
:103C5000D09033040E94E20B88579C4E909324042A
:103C600080932304F8018581811509F4C0C08D2D4E
:103C70008C298D79811190C0E114F0E5FF0608F5DB
:103C8000E11420E4F20608F09BC036EEE316F104DE
:103C900009F449C0C70190528115904208F097C0BD
:103CA000D80116968C91803108F46EC0C70199270F
:103CB000109238048D32910509F582E08093380422
:103CC0008AC0B0EEEB16B2E5FB0608F04DC0E0ECA2
:103CD000EE16E2E5FE0638F5F0EAEF16F2E5FF062D
:103CE000E8F420E6E21622E5F206E8F4C701925570
:103CF00080349105C0F010923804C7018E329105CE
:103D000008F082C08832910508F063C08E319105B9
:103D100008F061C004974A9780F23EC034EBE31686
:103D200032E5F30641F7D80115969C91911509F4F7
:103D300024C510922604970130572332310508F02C
:103D40002BC584E090E00E94783490939204809395
:103D50009104F701E150F047E232F10508F077C035
:103D6000E35CFA4C0C943A3349E7E4164CE7F4066A
:103D700030F457E7E5165CE7F506A8F6BCCF8BE70D
:103D8000E8168CE7F806CECF8F2D8F71843159F26B
:103D9000863161F4109238040E94821380913404B9
:103DA00090912504892B8093340421C00E948213B2
:103DB0008091340490912504892B80933404B3CFEF
:103DC000D80116968C91803108F070CFACCFC70126
:103DD0006FCF8A9709F780912504811531F0809182
:103DE000380492E08927809338040E94B111F801C9
:103DF0008581F701E851FC47E730F10508F093CFE2
:103E0000E15AFA4C0C943A338C34910521F38D32FB
:103E10009240E0CF26E241EE61EE0E941713CACC39
:103E200027E245EE65EEF9CF26E241EE60EEF5CFF2
:103E300027E245EE64EEF1CF26E241EE62EEEDCFF1
:103E400027E245EE66EEE9CF28E241E0EBCF809134
:103E50009104816080939104609191047091920427
:103E600084E090E00E94A6340E948B13A3CC809142
:103E70009204886080939204EFCF809191048260D5
:103E8000E9CF809191048460E5CF809191048860AE
:103E9000E1CF809192048160EDCF809192048260A5
:103EA000E9CF809191048061D5CF809191048062A7
:103EB000D1CF809191048064CDCF0E948B138091EB
:103EC00091048068C7CF809191048C60C3CF8091AA
:103ED00092048360CFCF809191048E7FBBCF80917D
:103EE0009204877FC7CF809191048D7FB3CF80915B
:103EF00091048B7FAFCF80919104877FABCF80916E
:103F000092048E7FB7CF809192048D7FB3CF809142
:103F100091048F7E9FCF809191048F7D9BCF809164
:103F200091048F7B97CF0E948B13809191048F77A0
:103F300091CF80919104837F8DCF809192048C7F6B
:103F400099CF80919104992782FF939590FB82F9F4
:103F500090FB83F97FCF80919204982F909590FBEE
:103F600080F990FB81F986CF90919104892F8F7B06
:103F700096FF80646FCF0E948B1390919104892FDC
:103F800097FB87F9805866CF61E08EE090E00E9451
:103F90008C3462CF60E0F9CF90919104892F8F7EAD
:103FA00094FF806157CF90919104892F8E7F90FF6D
:103FB000816050CF90919204892F877F93FF886012
:103FC00059CF89E2FCC389E2E4C3B7E7EB16BCE74B
:103FD000FB0609F054C081E00E942E0474C0827276
:103FE000F701E052F847EB30F10508F043C0EA5919
:103FF000FA4C0C943A3380912A0480FF0BC08E7FD8
:1040000080932A048AE294E0D7D9109229040E946E
:10401000FE07D0CB816080932A0461E08695869567
:10402000B8DAC8CB811521F0FDDAC4CB8115E1F3F4
:10403000EFDAC0CB811521F078DABCCB8115E1F342
:104040006CDAB8CB811521F083DAB4CB8115E1F3BA
:1040500074DAB0CB811521F091DAACCB8115E1F3A4
:1040600082DAA8CB811521F0DDD9A4CB8115E1F34B
:10407000CFD9A0CBE7E7EE16ECE7FE0609F1F8E7AB
:10408000EF16FCE7FF0629F19701205E324520324A
:10409000310520F5911122C02E2D2F7181E090E085
:1040A000AC0102C0440F551F2A95E2F77A01642F34
:1040B00083E090E00E948C348E2D0E941E047ACB07
:1040C00081E00E94240443E062E081E00E94C80491
:1040D00071CB82E0911509F47FCFF3CF4091320488
:1040E00080913704282F30E02095309570E024230C
:1040F0003723232B19F04823409332045BE7E5165E
:104100005CE7F50641F4911509F454CB0E940B04C9
:104110000E94800A4FCB80E4E81682E5F80608F09A
:104120005AC0A0E2EA16A2E5FA0608F05BC0E11464
:10413000B0E5FB0670F5E114E0E4FE0608F068C0A7
:10414000911509F47EC0BAE5EB16BCE7FB0609F44D
:10415000DAC008F0BCC0F1E0EF16FCE7FF0609F496
:10416000D0C023E0E2162CE7F20609F4C4C0E11443
:104170003CE7F30609F065C00E948B138FEF94E3D0
:10418000ACE081509040A040E1F700C000000E94E8
:10419000CF10970130552115324090F6970145E038
:1041A000369527954A95E1F7822F8F70209132043A
:1041B00030E041E050E0082E02C0440F551F0A9441
:1041C000E2F724233523232B09F4BACF9111A0CF92
:1041D00010923404F6C29701205C3245203231053A
:1041E00008F0AECF8E2D8F712091320430E041E087
:1041F00050E0082E02C0440F551F0A94E2F7242312
:104200003523232B09F49CCF911509F4D3CA80CF11
:10421000D80116968C91803108F092CF911111C07F
:104220002F2D2F7081E090E002C0880F991F2A95F2
:10423000E2F72091320430E082239323892B09F0A6
:10424000B9CAD80117968D919C91009709F45FC067
:104250000E9412067C01D8011596BC9015971696FF
:10426000AC90A2942FE0A22280913904877081152E
:1042700009F1CB2CB114F9F08F2D807F803469F0D7
:1042800080E28E0D8830B0F08F2D807E803229F450
:10429000B2E0EB1678F0A11469F08091920482FFED
:1042A00009C082E00E94F104809139048770CC2417
:1042B000C3948111C12CEF2DE295EF70F0ECFF1645
:1042C00008F09FC0F0E0EF58FA4C0C943A334BE5FD
:1042D000E4164CE7F406C9F080919204002482FFB2
:1042E0000394802D5CE5E5165CE7F50609F0A9CF9F
:1042F0000E944211A6CF6FEF7FEF80E090E00E9416
:10430000A6340E94B91381E0F3CF80E0F1CFF80129
:104310008581C080D180811569F0C6010E942C176B
:10432000F82E682FC6010E949204B6018F2D0E94BC
:1043300002178ECFC6010E94AD04F82EF6CF2F2DA6
:104340002F70D22E30E1F31618F0D29490EFD922CC
:10435000B114B9F0D11469F080E28E0D883010F0FC
:10436000E11009C0809134048D29809334040E94A7
:10437000B1118E2D44C0809138048D29809338046A
:10438000F6CF8E2D0E94A912D114D9F180E28E0DA4
:10439000883010F0E11004C08D2D0E940C0506C07D
:1043A000D094809138048D21809338040E94B111FB
:1043B00028C04F2D4F70D42E8F2D807F803219F062
:1043C000D29480EFD822E11451F051E0E51609F4BF
:1043D00083C0B11409F48FC0A114A9F1CACF809190
:1043E000920482FD2CC0B11421F1D11439F08091D6
:1043F00034048D29809334040E94B11180E00E941E
:104400000512C11409F4D9C08091390480FDD5C0CA
:10441000F80115828695869586950E942404C80128
:104420000AD9809139048695869586950E942E0436
:10443000C4C080E00E94A912D11419F3ADCFB11409
:1044400069F1A11004C08D2D0E940813DACF81E01C
:10445000A81210C0F09033048D2D8F21D81689F248
:104460000E94E20B90933D0480933C04FD28F0925F
:104470003304C7CF95E0A912C4CF8D2D0E94081335
:104480008D2D0E943C0C809135049D2D9823D916CA
:1044900009F4B7CF8D2980933504B3CFA11012C092
:1044A0008D2D0E9411138D2D0E943C0C809135049E
:1044B0009D2D9823911509F4A4CFD094D822D092A1
:1044C00035049FCFA1E0AA129CCF809134048D21A6
:1044D000811509F496CFE4CFB11429F0B6E0AB16FC
:1044E00008F08FCFB0CFE5E0AE1608F08ACF8D2D63
:1044F0000E94111386CFA114D1F3F9E3EF1209C082
:104500002FEF37EE43E0215030404040E1F700C04C
:1045100000008E2D0E94A91274CF8F2D869586954E
:104520008370811561F0813009F06BCFC701937002
:10453000B11002C080E090E00E94570B62CFC7012B
:104540009370B11002C080E090E00E942F0B59CF11
:104550006B2D8E2D0E947A0C54CF8F2D837081117C
:1045600039C0B11028C04E2D429546954770440F72
:10457000440F8E2D8F70042E01C0880F0A94EAF725
:104580002E2D2071E4FE07C02FE030E001C0220F85
:104590004A95EAF720953F2D36953695337032309F
:1045A000A1F0333081F040913604313059F0822B44
:1045B00084230E941E040E94200B60E0C8010E9418
:1045C000561708C9842B822BF4CF822B9091360486
:1045D0008927EFCFB11459F1F0FEEDCF4E2D429562
:1045E00046954770440F440F8E2D8F70042E01C0E6
:1045F000880F0A94EAF72E2D2071E4FE07C02FE001
:1046000030E001C0220F4A95EAF720953F2D3695FC
:1046100036953370323089F0333069F04091370489
:10462000313041F0822B84230E942104C4CF823098
:1046300010F2D4CF842B822BF7CF822B90913704AA
:104640008927F2CF5F2D5F70F52EB11439F0852FD9
:104650000E9424048E2D0E940813ADCF8E2D0E943F
:1046600011138F2D0E942E04A6CF82EFE816A1F120
:1046700093EFE91680F4A0EFEA16E1F0B1EFEB1644
:10468000A1F0B11409F467C0A11409F461C08E2D22
:104690000E94051290CFE3EFEE1629F1F4EFEF122E
:1046A000F0CF8091920482FD2AC08F2D8F71B114BA
:1046B000C9F216C0B11469F025E0A21608F07BCF4C
:1046C0002F2D2F7181E090E001C0880F2A95EAF725
:1046D000B5CF36E0A316F2CF8F2D8F71B110C2CFB8
:1046E0000E94240468CF80E0B11409F49DCF9F2D6F
:1046F0009F7181E001C0880F9A95EAF795CFB114B8
:10470000C1F0809139048770843049F410923904E3
:1047100010923B0410923A048F2D8F71A3CF45E085
:1047200063E0A41608F047CF8F2D8F710E94260CEE
:1047300042CF55E0A51640F01092390410923B0488
:1047400010923A0464E0F0CF81E00E94F10433CF8C
:104750008F2D8F71C5CFA114F9F289E3E81209C03A
:104760009FEFA7EEB3E09150A040B040E1F700C04A
:1047700000008E2D0E94A9121ECFB6E1EB16BCE7F9
:10478000FB0609F022CC80912704811509F41BCC8B
:1047900085E30E94B30B15C080913404E6E1EE1668
:1047A000ECE7FE0609F01BCC8A7A91E0811101C08A
:1047B00090E090932704811509F403CC85E30E94CF
:1047C0007F0B0E94B1110C94DA1BF3E7EF16FCE7A4
:1047D000FF0611F00C94711B80912204811509F4DD
:1047E000DEC90E9482130C94DA1B80918E04803102
:1047F00078F480918D04811559F0E0913F04209167
:104800003E04309189044091880459E02E1301C080
:1048100008956E2F70E05E9FF0011124DF01A05C0F
:10482000BB4F14968C911497811559F111968C9168
:104830001197831326C08C91841323C015968C91F5
:10484000159781111EC012968D919C91A0918A049A
:10485000B0918B048A1B9B0B883C910590F480914E
:104860008E048F70806180938E04EA5BFB4F8081A1
:104870008F708061808388E894E00E941B1B0C94F9
:10488000E704FB013196E770C1CFAFE0B0E0EBE4A5
:10489000F4E20C9467338C0186E0F801DE011A968D
:1048A00001900D928A95E1F7F801F580848198E8EE
:1048B000892E94E0992E60908C04611017C08115A8
:1048C00091F0F11409F417C1C8010E9485178115F0
:1048D00009F411C189E0F801A8E8B4E001900D9253
:1048E0008A95E1F782DFFF24F39456C07080A2809E
:1048F000B380D0908D0420918A0430918B04A5015F
:10490000421B530BD11409F4C6C0483C510508F0B2
:1049100079C0811541F380918904C180E0908E04B3
:1049200050E1E51608F059C0C81215C080918804FE
:10493000871111C0F1104BC08E2D8F708061809354
:104940008E0488E894E00E941B1B80918E04F8017D
:104950008683F12C21C0F1103AC040E06C2D872DE8
:104960000E948A1040E06C2D872D0E948A10F82E3C
:104970008111EFCF8A859B850E947817292F229578
:104980002F70903470F49F702230A0F09115B1F028
:10499000F8019681903190F48F2D2F96EEE00C94D3
:1049A00083332A5F2F70223068F0C8010E941B1BDE
:1049B000FD2CF2CF911511F0811571F3805E8830D6
:1049C00058F3F3CF803F40F3815F8330F9CF80917C
:1049D0008E04816080938E04BCCFC8123BC080914E
:1049E0008804871137C0F11035C0E682C8010E94E3
:1049F0001B1B89E0F801A8E8B4E001900D928A95AC
:104A0000E1F771CFE0908E04F0E1EF1650F488E802
:104A100094E00E941B1B89E0F40111928A95E9F74A
:104A200098CF811509F45FCF90918904F8018181B5
:104A3000981310C08091880487110CC0F1100AC02F
:104A4000E682C8010E941B1B89E0F40111928A953D
:104A5000E9F749CFC8010E948517811509F44BC0B9
:104A6000F11409F448C080918E04803208F432CFEA
:104A70001E821F821886198680918804909189046D
:104A80009A838983BC82AB826D82EF82CE010196CC
:104A90000E941B1B1FCF483C510508F0BCCF81155D
:104AA00009F421CFF11439F190918904818198138F
:104AB00018C080918804871114C080918E0480FDF5
:104AC00098CF803108F495CF8683807F803F09F4AA
:104AD0008DCF8681982F907F905F8F70892B8683F2
:104AE00085CFC8010E9485178111F4CE80918E0474
:104AF000816080938E04C8010E941B1BF4CEA1E24A
:104B0000B0E0E5E8F5E20C9471334C8F5D8F6E8F69
:104B10007F8F88A3192F99A3911110923804198EB1
:104B20001A8E1B8E86E0FE017C96DE015396019064
:104B30000D928A95E1F708A18091920482FF1FC02F
:104B40000E94E20B20913A0430913B04821B930BAC
:104B50008838934138F08091390482FD03C082E0A7
:104B60000E94F1040E94E20B20913C0430913D042C
:104B7000821B930B8838934110F00E941405011595
:104B800061F00F8B188F61E0CE0143960E9456179B
:104B900061E0CE0143960E9456170F8B188F89E073
:104BA000FE017396DE011A9601900D928A95E1F747
:104BB000CE010A966ADE811110C020913E04309128
:104BC0003F0489E0FE013A96DE01119601900D92B4
:104BD0008A95E1F78E8581110BC019E080913F0421
:104BE00090913E0489132BC0A196E4E00C948D3380
:104BF000822F90E00196877099273817190671F473
:104C00000E948B1310923E0410923F0489E0E8E862
:104C1000F4E0DF011D928A95E9F7DFCF99E0929FDA
:104C2000D0011124A05CBB4FFE01319601900D9282
:104C30009A95E1F780933E040E94E704CECF189F37
:104C4000C0011124805C9B4F20DE811569F28091A8
:104C50003F0490E001968770992780933F04BECF70
:104C6000A6E0B0E0E6E3F6E20C9471330E94E20BBA
:104C70008C0180918403909185038017910771F0D6
:104C800019821A820E94E20BBC0149815A8180E09C
:104C900090E035DF10938503009384032696E4E0CB
:104CA0000C948D33A6E0B0E0E8E5F6E20C947133A5
:104CB0008C019093810380938003011580E2180793
:104CC000B0F4C801805E9109089728F06FE673E19F
:104CD0000115110511F468E073E1C8010E94DC03BD
:104CE000802F0E9405122696E4E00C948D3380EF0D
:104CF00089838A830E94E20B8160BC0149815A81C9
:104D000081E091E0FCDEEFCFA6E0B0E0EAE8F6E279
:104D10000C9471338C01909381038093800301156F
:104D200080E21807B0F4802F0E94A912C801805EAB
:104D30009109089728F068E773E10115110511F44E
:104D400061E173E1C8010E94DC032696E4E00C9463
:104D50008D3380EF89838A830E94E20B8160BC01DE
:104D600049815A8181E090E0CADEEFCFA0E1B0E056
:104D7000ECEBF6E20C946533FE01319680E1DF0145
:104D80001D928A95E9F703E310E097EDA92EB12C67
:104D900029E2422E23E0522E612C712C4F01730127
:104DA0006201B1E14B165104610471041CF080E111
:104DB000C82ED12CA601B501C4010E947D34AC0CD3
:104DC000BD1C0D2C000CEE08FF084C185D086E0889
:104DD0007F080150104019F76096E0E10C94813390
:104DE0006FEF85E290E00E948C346FEF86E290E0F6
:104DF0000E948C346FEF87E290E00E948C3460E078
:104E000088E290E00E948C340E94C718AFDF6AE508
:104E100085E290E00E948C346CE986E290E00E948A
:104E20008C3465E687E290E00C948C348F929F92EC
:104E3000AF92BF92CF92DF92EF92FF920F93CF93F8
:104E4000DF9388E090E00E9473344B015C01CAE27A
:104E5000D4E068839982AA82BB821C821D821E8252
:104E60001F8283E290E00E946B34282F30E040E004
:104E700050E060E070E080E090E000E20E949A3351
:104E8000282939294A295B29288339834A835B8366
:104E90006C837D838E839F83DF91CF910F91FF90F1
:104EA000EF90DF90CF90BF90AF909F908F9008953C
:104EB000A3E0B0E0EEE5F7E20C946633FE01319634
:104EC00083E0DF011D928A95E9F78BE7E82E81E008
:104ED000F82E8F019EE7C92E91E0D92E3F01AA241A
:104EE000A394B12C33E8832E31E0932EF701819106
:104EF0007F018F3F09F43EC0F894E82FE295EF70F0
:104F0000F0E021A18F70A50102C0440F551F8A95C2
:104F1000E2F7CA01922F982B91A392A18095892341
:104F200082A3789400C0EEE7F1E031E0512C2191AA
:104F30002F3F79F0A22FA295AF70A05EB0E08C91C8
:104F400090E02F7002C0959587952A95E2F780FF33
:104F500036C080E0582A330F8E169F0641F7F701BE
:104F600082918F3F11F00E94100750EA5A95F1F795
:104F7000D8015C920F5F1F4FCE14DF0409F0B6CF4B
:104F800043E050E0B30184E692E00E944734892B6D
:104F9000C1F089819A81AB8180936402909365020C
:104FA000A093660281E080932C020E94E20B909312
:104FB0002B0280932A022396EFE00C948233832FF6
:104FC000C9CF80912C028115B1F300912A02109172
:104FD0002B020E94E20B801B910B059760F343E0CC
:104FE00050E064E672E08AE793E00E944734892B40
:104FF00061F08091640290916502A09166028093B5
:105000007A0390937B03A0937C0310922C02D3CF5E
:10501000CDB7DEB7E8970FB6F894DEBF0FBECDBFB1
:1050200085B7806885BF85B7806885BF1092AD025F
:105030001092AF021092AE0280EC8093720380EB6C
:1050400092E0909374038093730310927103109213
:10505000700310928D0210928C0210928F021092A7
:105060008E0210929102109290021092930210926E
:10507000920210929502109294021092970210924E
:105080009602109299021092980210929B0210922E
:105090009A0210929D0210929C0210929F0210920E
:1050A0009E021092A1021092A0021092A3021092EE
:1050B000A2021092A7021092A60281E39EE09093B2
:1050C00089028093880286EA9EE09093A9028093E9
:1050D000A8028AE297E09093A5028093A4028BE253
:1050E00097E090938B0280938A0284B7877F84BF76
:1050F0000FB6F894A8958091600088618093600055
:10510000109260000FBE80E890E00FB6F894809394
:105110006100909361000FBE81E080932D018EE0CD
:1051200097E090930102809300020E9489180E94E8
:10513000EA0D0E9430108091E20084608093E200CA
:10514000789480917F03811599F08091E900109106
:10515000EC008F70179511271795182B1092E90006
:105160008091E80083FD0E94CE131F701093E90028
:1051700082E084BD93E095BD9AEF97BD80936E0069
:105180000E94C817811101C02BDEEBE7F2E088E036
:10519000DF011D928A95E9F783E080937A0210E09F
:1051A00060E0812F0E94330A61E0812F0E94330A60
:1051B0001F5F1330A9F7EFE8F1E03197F1F700C076
:1051C000000010E080917A02181708F481C080EF87
:1051D0000E94100781EF0E94100784EF0E941007C1
:1051E0000EE711E093E8E92E91E0F92ED8018D91B8
:1051F0008D018F3F11F00E941007E016F106B1F704
:1052000083E0EAE7F3E0DF01282F1D922A95E9F712
:10521000E4E6F2E0DF011D928A95E9F780E090E094
:105220000E947834833E9E4F21F40E94C81781115A
:105230002AC063EE7EEF80E090E00E94A63460E03A
:1052400082E090E00E948C3481E08093360461E03B
:1052500083E090E00E948C3460E074E184E090E0B0
:105260000E94A6340E94FD19BBDD40E050E0BA0167
:105270008FE090E00E949E3440E050E0BA0183E16C
:1052800090E00E949E3482E090E00E946B34809314
:105290006A0284E090E00E947834909392048093B4
:1052A000910406DEEFEFF6E721E0E150F040204008
:1052B000E1F700C00000FCDD80917A0380FF1AC096
:1052C0006FEF7FEF80E090E00E94A6340E94CF1045
:1052D00060E0812F0E94560A082F61E0812F0E9412
:1052E000560AE12FF0E0E958FD4F880F802B8083AC
:1052F0001F5F68CF83E090E00E946B340E941E0421
:105300008091670281111EC08AE294E08FDD809156
:105310002A04843028F40E94FD198AE294E086DD94
:105320000E94F007109229040E94730A80912A04B7
:1053300080FF05C060E0869586950E94C91A81E0CD
:105340008093670282E191E09093A7038093A60384
:105350008E010F5F1F4F80917F03853069F4B0E4A9
:10536000FB2E82E1E82E80917F03853009F484C012
:105370000E948B130E94200B9BDD90916B02809109
:105380007A039813C8C090916C0280917B039813A4
:10539000C2C090916D0280917C039813BCC060DC08
:1053A00080912204811569F00E94E20B2091230470
:1053B00030912404821B930B8F3F9F4710F40E946F
:1053C000821380912904811509F446C08091280434
:1053D000E0912A04E695E695E81BE093700285319A
:1053E00009F440C108F0E3C0893009F42FC108F086
:1053F000CFC0823009F414C1863009F41CC170EDAD
:10540000E72E77E0F72EE9E2CE2EE7E0DE2E809160
:105410007102811561F0109271020E94E20B90936B
:105420006F0280936E0210927302109272020E94B9
:10543000E20B20916E0230916F02821B930B8F3F23
:105440009F4750F42E0D3F1D30936F0220936E0244
:105450008EE692E0F601099580918302811551F064
:1054600080917D021092830280937E0280917B0264
:1054700080937C02E12C4BC180917F03843019F131
:105480001092680288E190E00FB6F894A895809396
:1054900060000FBEF092600083B7817F846083BF9D
:1054A00083B7816083BF7894889583B78E7F83BFED
:1054B0000FB6F894A8958091600088618093600091
:1054C000109260000FBEF4DC80917B0390917A0310
:1054D000892B90917C03892B811509F444CF80910D
:1054E0006902811509F43FCF90E199BDE9BC09B487
:1054F00000FEFDCF8091D8008F7D8093D8008091F1
:10550000E00082608093E0008091E00081FDFCCFAC
:105510000E948B1328CFFAE7CF2EF3E0DF2EABE605
:10552000EA2EA2E0FA2EB12CD601AD906D01F70162
:1055300081917F018A1529F1782E7A24912C882473
:105540008394872D88218115A9F09982BA820E94BF
:10555000E20B9C838B83F1E0FD8391E08A2D88210F
:10556000811101C090E09E8349815A816B817C81C9
:105570008D81C5DA9394880C25E09212E2CFF70171
:10558000A292B39433E0B312CFCF0E94350D08CF6F
:105590008F3009F034CFE695F0E0E051FA4FE49116
:1055A000EE2EF12C34EAC32E38E0D32E30CFA4EF08
:1055B000EA2EFF24F394B6ECCB2EB9E0DB2E843236
:1055C00009F425CFB0F4E8E2EE2EF12CF6E4CF2E6C
:1055D000F9E0DF2E883109F41ACF833209F00FCFBA
:1055E000EBEEF5E0E590F59091E3C92E98E0D92E29
:1055F0000ECF853209F003CF8BEAE89F812D11246D
:10560000982F96958E7F890FE81BF0E0E851FA4FAE
:10561000E491EE2EF12C8BE4C82E89E1D82EF7CE42
:10562000F0E0E750FA4FE491EE2EF12C6BE6C62E37
:1056300068E0D62EECCEF0E0EA50FA4FE491EE2E80
:10564000F12C5CE5C52E58E0D52EE1CEE695F0E0D4
:10565000ED50FA4FE491EE2EF12C4EE7C42E48E0C7
:10566000D42ED5CEF0E0E351FA4FE491EE2EF12C9A
:105670002EEFC22E28E0D22ECACE61E08E2D0E94DF
:10568000560AC82E60E08E2D0E94560ACC0C8C293A
:105690002E2D30E0D901A958BD4FEC919E2F93706B
:1056A0008917A1F1EE0FEE0FE82BEC93EF70F0E00D
:1056B000ED57FE4F2C583D4F8081D9019C91890FA9
:1056C0008C9384300CF455C04F2D50E0BA016F5FBD
:1056D0007F4F63707727D616170681F045585D4FC8
:1056E0009E2D9F77FA01948391E09F0D9370909384
:1056F0007D0290917B029F5F90937B02082E000CAD
:10570000990B64E070E0A3D7F9018083E394D09013
:105710007E02F0907D0280917A02E81608F4ADCF07
:1057200090E06CEFE62E7DEFD72E80917E022091E7
:105730007D02281709F457C0E82FF0E0E158FD4F2B
:10574000908197FBCC24C0F8F92EE894F7F88F5F8E
:10575000837080937E0280917C028F5F80937C02B5
:1057600097FD1CC0F9A6EAA60E94E20B43E0B42E06
:105770001BC08D3F1CF64F2D50E0BA016F5F7F4F6D
:1057800063707727D616170609F4B8CF45585D4FD2
:105790009E2D9068DA0114969C93A6CFF9A6DAA6FE
:1057A0000E94E20B52E0B52EBC018BA79CA7BDA6C0
:1057B000F1E0FEA749A55AA58B2D91E0A0D9FFA63F
:1057C000C11479F0D8AA0E94E20BBC0189AB9AAB54
:1057D000BBAA1CAA4FA558A98B2D90E090D991E0A7
:1057E000A4CFE8AAF0CF91110E94350D86E0ECEB32
:1057F000F3E0D80101900D928A95E1F79090BD03F6
:10580000D090BE03B090BF03A090C003C090C1036E
:105810001092BE031092BF031092C0031092C103F6
:105820008D2D8B29811509F441C0E0908602F090FE
:1058300087020E94E20B9C012E193F099091BA0346
:10584000911509F460C52531310580F19F3F19F0AC
:105850009F5F9093BA03D11459F00E94B50A91E06A
:105860001D140CF09FEF899F802D11248093BE039F
:10587000B11459F00E94B50A91E01B140CF09FEF8F
:10588000899F802D11248093BF038091BE038115D1
:1058900069F0F090BF03F11449F00E94A70A8093C9
:1058A000BE038F2D0E94A70A8093BF038C2D8A29E7
:1058B000811509F441C0E0908402F09085020E94B5
:1058C000E20B9C012E193F099091B903911509F43F
:1058D00015C52135310580F19F3F19F09F5F9093E9
:1058E000B903A11459F00E94D50A91E01A140CF0E2
:1058F0009FEF899F802D11248093C003C11459F01C
:105900000E94D50A91E01C140CF09FEF899F802D16
:1059100011248093C1038091C003811569F0F09038
:10592000C103F11449F00E94A70A8093C0038F2D90
:105930000E94A70A8093C1038091BD03891119C0F9
:105940008091BE03811511F0D81213C02091BF03BE
:10595000211511F02B110DC09091C103911511F07B
:10596000C91207C03091C003311103C0822B892BAB
:1059700081110E94510C86E0F801ACEBB3E001907C
:105980000D928A95E1F7E091A802F091A902309773
:1059900019F088E892E009959FB7F894E0907103B8
:1059A00080917003E81608F472C0E81A9FBFC12CFA
:1059B000D12CF12CAA24A394B12CCE14DF0408F42A
:1059C0006AC00E94200B90917503891721F0809383
:1059D00075030E94350D80917F038430E1F480913E
:1059E0001F018F708093E9009091E80090FF13C031
:1059F00090917F03943079F48093E9009091F300C3
:105A00008091F200892B39F08091E8008E778093A5
:105A1000E8000E94B90D80917F03843009F09BCC8F
:105A200083E08093E9008091E80082FF94CC80912C
:105A3000E80090E085FF08C040E050E060E270E0E0
:105A4000C8010E947E0E91E08091E8008B778093E0
:105A5000E800911509F47FCCE0908203F090830375
:105A6000E981E114F10409F4CCC0EE3F09F0ECC087
:105A70008A81833020F08550833008F0E5C0EA81C8
:105A8000EE3008F0E1C0F0E0E358FA4CF3C52091A5
:105A90007203E20E8ACF8091700390E060917203EE
:105AA00070E0D5D52091730330917403280F391F0E
:105AB000D9019C908090AD02B8EF9B16E8F0E1E030
:105AC000E093AD0220E040E0692D81E090E00E948B
:105AD000280F8092AD022FB7F8948091700390E068
:105AE00001966091720370E0B2D5809370032FBF6E
:105AF0008FEFC81AD80A61CF97FE53C0F4E08F1613
:105B000031F09092AA02B092AF02A092AE02892D1B
:105B10000E942C07823081F0833071F0813079F45B
:105B20008093AD0220E040E0692D81E090E00E948A
:105B3000280F1092AD02CFCF8093AD02CCCF20EFD3
:105B4000921651F037EF931699F01092AD02109221
:105B5000AF021092AE02BFCF84E08093AD0290926C
:105B6000AA0281E090E09093AF028093AE02B3CF9F
:105B70002091AE023091AF02C90163E070E053D5CD
:105B8000FC01E857FD4F92A2C90101969093AF0224
:105B90008093AE022091AC024091AB026091AA02C8
:105BA000C6CF811409F497CF2091AE023091AF0295
:105BB000C90163E070E037D5AC01FC01E857FD4F47
:105BC00092A2C90101969093AF028093AE02413038
:105BD000510591F04230510509F07DCF2091AC0282
:105BE0004091AB026091AA020E94280F8091AD0201
:105BF000843009F0B6CF6FCF42E020E084126BCF43
:105C0000EFCFE43148F4E11551F0E150E33138F4DD
:105C1000F0E0E557FA4C2EC5EE3F09F430CF8FEF98
:105C2000898312C01A8289E08B830EC08A818230F8
:105C300079F08330A9F0813091F70E94350D30D58D
:105C40006B837C838D839E83C8010E941A0F83CB54
:105C500088E290E040D61B821C821D828E83F4CFA6
:105C600080917D0390917E03892B71F380917A035B
:105C70008B8380917B038C8380917C038D83E4CF25
:105C80008A81823061F66B817C818D819E8108D50D
:105C900088E290E041D6D8CF4C816B818A810E9406
:105CA0009B169827892798279E838D83CDCF2D819A
:105CB0003E813227232732274C816B818A810E94C3
:105CC0005911C2CF0E94C718BFCF8A81823891F183
:105CD000B0F48038E9F0813809F0B6CF60E08B810C
:105CE0000E94C91A9B8180912A0491111AC08E7F4B
:105CF00080932A04109229040E94FE07A5CF8338BE
:105D000009F0A2CF20E040912D046C818B8106C068
:105D100020E04B8160912C0480912B040E941C1A7E
:105D200093CF816080932A0460E0869586950E94D7
:105D3000C91A8ACF8B8180932E0486CF8A818238BC
:105D4000E1F060F48038A1F0813809F07DCF8091D6
:105D50002A0480FF10C08695869566CF833809F0A7
:105D600073CF80912B048B8380912C048C836CCF18
:105D700080912D0459CF80E057CF80912E0454CFCD
:105D80000E94F0078AE294E00E94DC195DCF80E176
:105D90008A835ACF83E08A8389E246CF8C818D3112
:105DA00008F052CF8A809B80982489249824A12CC3
:105DB000B12C78016801C80ED11CCE14DF0409F49F
:105DC00043CF80E099E2891693E09906A104B104DB
:105DD00020F4C40189529F4F7ED5D70114968C932D
:105DE000BFEFEB1AFB0AEFEF8E1A9E0AAE0ABE0A4D
:105DF000E4CF80917D0390917E03892B09F424CF19
:105E00008C818D3108F020CF482E512C612C712CC3
:105E1000CA80DB80DC24CD24DC24E12CF12C1801A9
:105E2000812C912C540184149504A604B70408F025
:105E30000BCFF9E2CF16F3E0DF06E104F10438F40A
:105E4000D10114966C91C60189529F4F65D5BFEF61
:105E50008B1A9B0AAB0ABB0AEFEFCE1ADE0AEE0AD8
:105E6000FE0AFFEF2F1A3F0ADECF0E94B626ECCEC5
:105E700083E08ECF8C818D3108F0E6CE482E512CF8
:105E8000612C712CCA80DB80DC24CD24DC24E12C45
:105E9000F12C812C912C54011E0125E0220E311C85
:105EA00084149504A604B70408F0CECE80E03AE549
:105EB000C316D104E104F10418F4C60189960BD588
:105EC000D1018D931D01BFEF8B1A9B0AAB0ABB0A50
:105ED000EFEFCE1ADE0AEE0AFE0AE2CF2C81E22EA6
:105EE000F12C2D3108F0B0CE8A819B81982789272B
:105EF00098272C01612C712C8A35910508F0A4CECD
:105F0000822E912CA12CB12C4AE550E060E070E08B
:105F1000441955096609770942175105610571054C
:105F200008F492CE20917D0330917E03232B09F05B
:105F30003FC09C01275D3F4F38AF2FAB80FBCC2487
:105F4000DD24C0F880FF0BC08896C5D49D818927C9
:105F50009827892781159C4711F48FEF8D83D501F0
:105F6000C401840D951DA61DB71D80FF1AC0170121
:105F700041E0241A3108CE010596820D931D9EAB97
:105F80008DAB8FA998AD8E0D9F1DA5D4ADA9BEA9CF
:105F90009C9181159C4721F48FEFEDA9FEA9808388
:105FA0007101F801EC0DFD1D2FEFCE14DF0428F078
:105FB0001801C12CD12C760125C0948185818115D1
:105FC0009C4711F42483258342E0C40ED11C3296F1
:105FD000ECCF8AE5481651046104710430F4D10114
:105FE00014966C91C201899697D4BFEFCB1ADB0A45
:105FF000EB0AFB0AEFEF4E1A5E0A6E0A7E0AFFEF0B
:106000002F1A3F0AC814D904EA04FB0410F31CCE6B
:1060100080917D0390917E03892B09F415CEC801F0
:106020000E941A0F2FEF31EE44E0215030404040E3
:10603000E1F700C000004AC988E0EEE2F1E0DE01CD
:10604000919601900D928A95E1F7FE0132968FE1CB
:10605000DF011D928A95E9F786E0898388E07F96C3
:10606000DE01159601900D928A95E1F7EDCD88E15C
:10607000898381E08A831B821C82E6CD8B819C818F
:10608000092E000CAA0BBB0B25E0880F991FAA1F35
:10609000BB1F2A95D1F7AC01BD01405E5F4F6F4F2A
:1060A0007F4F481759076A077B0708F4CDCD883121
:1060B000E1E09E07A105B10508F0C6CD4931F1E048
:1060C0005F076105710520F048E151E060E070E094
:1060D000481B590BBC0163507A4FC801C2D3B4CDE1
:1060E000FB80EC8040E06E2D8F2D0E94CA16982711
:1060F000892798279A83898341E06E2D8F2D0E94EE
:10610000CA169827892798279C838B839DCD2E813B
:106110003F812C37310569F032272327322741E0B0
:106120008D81811101C040E06C818B810E948011C2
:106130008BCD80917D0390917E0320E03CE7892BFD
:1061400071F720E030E0EBCF4AE150E06FEF70E014
:10615000CE010796A9D380917D038983EA821B82B1
:1061600082E08C831D8283E079CD81E090E0909382
:1061700083038093820382E390E09093790380937A
:1061800078030E94E20B90937703809376035CCDB3
:10619000E114F10471F1B0907A03C0907603D090CD
:1061A00077030E94E20B8C199D098536910540F119
:1061B000B3FE26C0B2FE24C00E94E20B9093770388
:1061C000809376038091780390917903019790935F
:1061D000790380937803892B61F4109283031092E2
:1061E000820381E090E090937E0380937D03E12C15
:1061F000F12C80917D038983EA828091780314CD0C
:1062000082E390E09093790380937803F2CF109229
:106210007E0310927D0318CD40E250E06FEF70E0F6
:10622000C80142D311CD8B81873071F0883049F19C
:1062300081110ACD8FE1D8011D928A95E9F788E096
:106240008C8383E088A300CD2C8166E0CE0181960B
:10625000FC01362F11923A95E9F7283080F4629FBD
:10626000B001112469557F4F46E050E024D380E00F
:10627000898386E0FE01B196DE011296F3CE8FEFA0
:10628000F7CF6C8186E0FE013596DE019196019094
:106290000D928A95E1F789A19AA181154CE794079F
:1062A00041F420917D0330917E03232B11F480E093
:1062B00090E09AA389A38BA19CA18115ACE79A07D2
:1062C00041F420917D0330917E03232B11F480E073
:1062D00090E09CA38BA38FEF683060F4B6E06B9FD7
:1062E000B001112469557F4F46E050E0CE01819600
:1062F00031D380E089830E948918A6CC2B303105E8
:1063000008F0ECCA19CB2B30310508F0A1CACECA6F
:106310001F921FB61F9211248F939F93AF93BF9329
:1063200080916802811113C08091420290914302D2
:10633000A0914402B09145024196A11DB11D8093E8
:10634000420290934302A0934402B0934502BF914E
:10635000AF919F918F911F901FBE1F9018957894B9
:106360001F921FB61F9211248F939F93AF93BF93D9
:106370008091420290914302A0914402B091450263
:106380000196A11DB11D8093420290934302A093F8
:106390004402B0934502BF91AF919F918F911F909E
:1063A0001FBE1F9018951F920F920FB60F921124C7
:1063B0002F933F934F935F936F937F938F939F930D
:1063C000AF93BF93EF93FF938091E10082FF09C0E9
:1063D0008091E20082FF05C08091E1008B7F809375
:1063E000E1008091DA0080FF24C08091D80080FF16
:1063F00020C08091DA008E7F8093DA008091D900EE
:1064000080FFA9C080E189BD82E189BD09B400FE99
:10641000FDCF81E080937F0380913102811109C01B
:106420000E94EA0D0E9430108091E2008460809307
:10643000E2008091E10080FF1AC08091E20080FFBD
:1064400016C08091E2008E7F8093E2008091E2008E
:1064500080618093E2008091D80080628093D800B0
:1064600019BC85E080937F0383E080932D018091A8
:10647000E10084FF2FC08091E20084FF2BC080E107
:1064800089BD82E189BD09B400FEFDCF8091D800AD
:106490008F7D8093D8008091E1008F7E8093E10012
:1064A0008091E2008F7E8093E2008091E200816023
:1064B0008093E20080913002811509F452C084E09B
:1064C00080937F0380917F03843009F052C082E083
:1064D00080932D018091E10083FF2CC08091E20028
:1064E00083FF28C08091E100877F8093E10082E0F4
:1064F00080937F03109230028091E1008E7F809321
:10650000E1008091E2008E7F8093E2008091E200C2
:1065100080618093E20042E060E080E00E94001031
:106520008091F00088608093F00081E080932D01DD
:1065300080932C01FF91EF91BF91AF919F918F912B
:106540007F916F915F914F913F912F910F900FBE6F
:106550000F901F90189519BC10927F031092310272
:1065600068CF8091E30087FF02C083E0A9CF81E07C
:10657000A7CF81E0ADCF1F920F920FB60F921124DB
:10658000EF92FF920F931F932F933F934F935F933D
:106590006F937F938F939F93AF93BF93CF93EF931B
:1065A000FF9309EE10E0F8018081C091EC008F703C
:1065B000C795CC27C795C82B108280EFE82EF12C09
:1065C000F7018081877F808378940E94CE13F80141
:1065D0001082F701808188608083CF70F801C083CA
:1065E000FF91EF91CF91BF91AF919F918F917F914B
:1065F0006F915F914F913F912F911F910F91FF905C
:10660000EF900F900FBE0F901F90189587FB082EEC
:10661000062687FD819567FD6195C2D00EF49195A0
:1066200007FC81950895AA1BBB1B51E107C0AA1F57
:10663000BB1FA617B70710F0A61BB70B881F991F23
:106640005A95A9F780959095BC01CD01089597FBC7
:10665000072E16F4009406D077FD08D0E4DF07FC7F
:1066600005D03EF4909581959F4F08957095619562
:106670007F4F0895EE0FFF1F0590F491E02D0994D0
:10668000082E817006940694811D0694811D06943F
:10669000811D0694811D0694811D0694801D089518
:1066A0006927962769277827872778270895B7D1FC
:1066B000332312F48A1B9B0B01C0B1D1B7FF08959D
:1066C000821B930B08952F923F924F925F926F928D
:1066D0007F928F929F92AF92BF92CF92DF92EF9272
:1066E000FF920F931F93CF93DF93CDB7DEB7CA1BF3
:1066F000DB0B0FB6F894DEBF0FBECDBF09942A881E
:10670000398848885F846E847D848C849B84AA84C5
:10671000B984C884DF80EE80FD800C811B81AA8152
:10672000B981CE0FD11D0FB6F894DEBF0FBECDBF1D
:10673000ED010895002E083090F0982F872F762FC6
:10674000652F542F432F322F22270850F4CF220FCA
:10675000331F441F551F661F771F881F991F0A95F7
:10676000B2F7002D089597FD1094002E083098F090
:106770000850232F342F452F562F672F782F892F1E
:10678000912DF4CF159497958795779567955795A3
:106790004795379527950A95AAF71124002D089556
:1067A000992778E0880F991F961708F0961B881F85
:1067B0007A95C9F7809508958F929F92AF92BF9274
:1067C000CF92DF92EF92FF92CF93DF93EC0168813B
:1067D00079818A819B81611571058105910521F47B
:1067E00064E279ED8BE597E02DE133EF41E050E095
:1067F000C8D049015A019B01AC01A7EAB1E4DDD040
:106800006B017C01ACEEB4EFA5019401E2D0DC0198
:10681000CB018C0D9D1DAE1DBF1DB7FF03C00197A1
:10682000A109B04888839983AA83BB839F77DF91AE
:10683000CF91FF90EF90DF90CF90BF90AF909F905F
:106840008F900895B9CF80E091E0B6CFA0E0B0E09E
:106850008093000190930101A0930201B093030182
:106860000895FB01DC0102C005900D92415050409B
:10687000D8F70895FC014150504030F001900616C1
:10688000D1F73197CF010895882799270895FB0103
:10689000DC0104C08D910190801921F441505040D9
:1068A000C8F7881B990B0895DC0101C06D93415016
:1068B0005040E0F70895DC01CB01FC01F999FECFCF
:1068C00006C0F2BDE1BDF89A319600B40D92415078
:1068D0005040B8F70895F999FECF92BD81BDF89A5E
:1068E000992780B50895A6E1B0E044E050E0E5CFF7
:1068F000A8E1B0E042E050E0E0CFDC01A40FB51F1A
:106900004150504040F0CB01840F951F2E9105D08F
:1069100041505040D8F70895262FF999FECF92BDE7
:1069200081BDF89A019700B4021639F01FBA20BD54
:106930000FB6F894FA9AF99A0FBE08950396272F86
:10694000ECDFEADF252FE9DF242FE7CF0196272FA1
:10695000E4DFE2CFDC01CB0102C02D9105D0415034
:106960005040D8F70895262FF999FECF1FBA92BD4F
:1069700081BD20BD0FB6F894FA9AF99A0FBE019620
:106980000895052E97FB16F400940FD057FD05D0FF
:1069900024D007FC02D046F408C0509540953095AD
:1069A00021953F4F4F4F5F4F08959095809570957B
:1069B00061957F4F8F4F9F4F089531D0A59F900DC8
:1069C000B49F900DA49F800D911D11240895B7FFD1
:1069D000F4CFF3DF821B930B0895A1E21A2EAA1BBA
:1069E000BB1BFD010DC0AA1FBB1FEE1FFF1FA2177F
:1069F000B307E407F50720F0A21BB30BE40BF50B7C
:106A0000661F771F881F991F1A9469F76095709504
:106A1000809590959B01AC01BD01CF010895A29F87
:106A2000B001B39FC001A39F700D811D1124911D62
:106A3000B29F700D811D1124911D0895F894FFCF10
:106A4000860C8B0C8D0C920CA20CA20CA20CA20C2E
:106A5000A20CA20CA20CA20C940C980C9B0CA00CE7
:106A6000B00CB60CBA0CAB14D114D714D114D71483
:106A700029154A15D71451165E166B1FD31F731FA5
:106A80003D1F411F771F451F7B1F871F511FCC1FB5
:106A9000551F8B1F591F8F1FB41F5D1F931FBB1FD7
:106AA000631F991FA11F491F7F1F4D1F831F671F52
:106AB0009D1FAB1FC41FCA1F371F6F1FDA1F141F74
:106AC000181F0A1F101F1C1F201F241FFB1F12202E
:106AD00016201A201E20222026202A202E20322096
:106AE00036209F219F21D921D9218D22A822012240
:106AF0000122AD222223352335231C3037303E308E
:106B000070308730A430B530C83007310C31242EB6
:106B1000242E242E1331122E162E402E4C2E572E9C
:106B2000622E652E9E2EC02E0F2E0830C72ECA2E26
:0C6B3000CE2EF92E352F382F3A2F6E2F65
:106B3C000100000001010201191A1B1C1D1E1F205F
:106B4C002122DF0B1D11331138113D111411048555
:106B5C004000000106400000010000000100B5A843
:106B6C003A61864595DF004422B684016201AC008F
:106B7C008A02A302C30236349635979400010202AE
:106B8C0002020606060909090909090F0F0F0F0F62
:106B9C000F15151518191919191919191919192366
:106BAC002425252525252503010203F0F1F4F5F60E
:106BBC00F7676600FF0100010000FFFF0000010005
:106BCC0001FF00E200E900EA00B500B600B700CD15
:106BDC00008301CC008A019201940121022302243A
:106BEC00022502260227022A02B300B4006F0070AD
:106BFC00009F01CB019F02A002E200E900EA00B570
:106C0C0000B600B700CD008301CC008A019201943C
:106C1C00012102230224022502260227022A02B3A2
:106C2C0000B4006F0070009F01CB019F02A0020016
:00000001FF
